:1000000096C40000CCC40000CAC40000C8C40000EC
:10001000C6C40000C4C40000C2C40000C0C40000C4
:10002000BEC40000BCC400000C9444300C942C31BD
:100030000C94F92FB4C40000B2C40000B0C4000096
:10004000AEC40000ACC40000AAC40000A8C40000F4
:10005000A6C400000C942030A2C40000A0C400007C
:100060009EC400009CC400009AC4000098C4000014
:1000700096C4000094C4000092C4000090C4000024
:100080008EC400008CC400008AC4000088C4000034
:1000900086C4000084C4000082C4000080C4000044
:1000A0007EC400007CC400007AC400000501098001
:1000B000A101850319012AB700150126B700950192
:1000C00075108100C0050C0901A101850419012AE0
:1000D000A002150126A002950175108100C005013E
:1000E0000906A1018506050719E029E71500250184
:1000F0009508750181020507190029EF15002501F2
:1001000095F075018102050819012905950575010C
:100110009102950175039101C00660FF0961A1017B
:100120000962150026FF00952075088102096315F4
:100130000026FF00952075089102C005010906A15F
:1001400001050719E029E7150025019508750181CA
:10015000029501750881010507190029FF15002680
:10016000FF0095067508810005081901290515008D
:100170002501950575019102950175039101C00056
:10018000000000000000000000000000000000006F
:10019000000000000000000000000000000000005F
:1001A0000000007E0F00D4FFFFFFC70000007800B2
:1001B000000000000000002A2B28000000000000C2
:1001C0000000000000000000000029000000002CDA
:1001D0001E3420212224342627252E362D37382779
:1001E0001E1F202122232425263333362E37381F85
:1001F0000405060708090A0B0C0D0E0F1011121347
:100200001415161718191A1B1C1D2F3130232D35E4
:100210000405060708090A0B0C0D0E0F1011121326
:100220001415161718191A1B1C1D2F3130354C09BF
:10023000025B00030100A0FA0904000001030101B0
:100240000009211101000122440007058103080073
:10025000010904010002030000000921110100014D
:100260002222000705820320000107050303200066
:10027000010904020001030000000921110100012D
:10028000226D000705840320000112010002000016
:100290000008504B01060100010203011C03760017
:1002A000690061006C003A006600360034006300AB
:1002B000320062003300630000001603580054004F
:1002C000360030005F00530049004E0047004100F7
:1002D000000012036B006F0070006900620065008F
:1002E0006E006700000004030904167C1E001F0056
:1002F00020002100220023002400250026002700E2
:100300002D002E002A002B0014001A0008001500F2
:1003100017001C0018000C00120013002F00300002
:100320002A00390004001600070009000A000B002B
:100330000D000E000F003300340031002800E100F2
:1003400064001D001B0006001900050011001000CC
:10035000360037003800E5002252E000E300E200FA
:1003600000002C0000002C0000002C000000225295
:10037000E6002152E40001003A003B003C003D0051
:100380003E003F0040004100420043004400450061
:1003900001000100010001000100007C01000100DA
:1003A0000100010001000100010001000100010045
:1003B0000100010001000100010001000100010035
:1003C0000100010001000100010001000100AA007C
:1003D000A900AE00AC00AB0001000100010001006B
:1003E0000100010001000100010001000000010006
:1003F00000000100000001000000010001000100F8
:1004000001000100010001000100010001000100E4
:1004100001000100010001000100010001000100D4
:1004200001000100010001000100010001000100C4
:1004300001000100010001000100010001000100B4
:1004400001000100010001000100010001000100A4
:100450000100010001000100010001000100010094
:100460000100010001000100010001000100010084
:100470000100010001000100000001000000010076
:100480000000010000000100010001000100222322
:10049000252628292A2C2D2F3032333536383A3B61
:1004A0003D3E4042434547494A4C4E5051535557B3
:1004B000595A5C5E6062646668696B6D6F717375D2
:1004C00077797B7D7F81838587898A8C8E909294D2
:1004D00096989A9C9E9FA1A3A5A7A8AAACAEAFB1DF
:1004E000B3B4B6B8B9BBBCBEBFC1C2C3C5C6C7C929
:1004F000CACBCCCDCED0D1D2D2D3D4D5D6D7D7D8E3
:10050000D9D9DADADBDBDBDCDCDCDCDCDDDDDDDD34
:10051000DCDCDCDCDCDBDBDBDADAD9D9D8D7D7D63C
:10052000D5D4D3D2D2D1D0CECDCCCBCAC9C7C6C5F3
:10053000C3C2C1BFBEBCBBB9B8B6B4B3B1AFAEAC39
:10054000AAA8A7A5A3A19F9E9C9A98969492908EE4
:100550008C8A89878583817F7D7B79777573716FBD
:100560006D6B6968666462605E5C5A595755535199
:10057000504E4C4A4947454342403E3D3B3A38364F
:10058000353332302F2D2C2A292826252322FFAA65
:100590007F55400001010101010101010102020238
:1005A000020202020202030303030303030304041F
:1005B00004040404040505050505060606060607E9
:1005C0000707070708080808090909090A0A0A0BA2
:1005D0000B0B0C0C0C0D0D0D0E0E0E0F0F0F101043
:1005E00011111112121313141415151616171718CA
:1005F0001819191A1A1B1B1C1D1D1E1E1F20202135
:100600002222232424252626272829292A2B2C2D7B
:100610002D2E2F30313232333435363738393A3B9C
:100620003C3D3E3F404142434445464748494A4C91
:100630004D4E4F50515354555658595A5B5D5E5F5D
:10064000616264656668696B6C6D6F7072737577F3
:10065000787A7B7D7E8082838587888A8C8E8F9155
:10066000939596989A9C9EA0A2A3A5A7A9ABADAF7F
:10067000B1B3B5B7BABCBEC0C2C4C6C9CBCDCFD169
:10068000D4D6D8DBDDDFE2E4E7E9EBEEF0F3F5F812
:10069000FAFDFF643214783C1E1E140A05FD377AF9
:1006A000585A000004E6D6B44602002101160000A4
:1006B00000742FE5A3E0085002285D003D8889C63C
:1006C0005436C3174FE4E9115795175DC3B323811F
:1006D0004B6A54FD087B10DA36ECAD99669996B3F7
:1006E00097B1EE56C9F0486B4C37A4DB201BD20AF9
:1006F0003C30A106E134E92CF3F1334E55B61D59D7
:100700002ABB30D775A9D9D17A0995C099FBD16A8E
:10071000429FDA868518E83AABD3D743152EE9DF36
:10072000A369361F3C40A35EE9BE547C9FAF94375B
:10073000332E9CC0F2AD79692FFB3D171A5AFDBBD1
:10074000EF08A50E9A30842C7247197A4355B917D1
:100750007EDA290A04D2183C3C1A20491866147221
:10076000E50F9B9E528657504039CC657E08F84B6A
:1007700032E5074F623A37CCFCF0F10F0B9E4798F9
:10078000C79763077FD42D78B956AE4575ECC34043
:10079000ED3080E9FBFD5C2607B2CBB194E746382B
:1007A0006DAC8EA1D43F9E5F7E6C0641944D3EC4DD
:1007B0009BE80D05731D353A42932AAC452BAC528C
:1007C000A783E6DFD142F4D4292E5138BE3CA1DC08
:1007D00074F27B54BBFFB57D8656634B1178DE6A9D
:1007E000194B1E9AB3FB14A8FD376AA8D7F8A6FBCD
:1007F0005EF95FC4E006820A3BCF2DA599D8602937
:1008000033CE558D2859BC90B2C12D581D90662904
:10081000A0EA65F89A27119DC1279D86D5015BFD49
:100820006D46C18EDA184E29C44FD271D6408E4D16
:1008300059EDC95E52030014079B97E5C3F5808903
:10084000AE966273846E487584C9E99E9CD4EDC0EF
:10085000A278562C8BDBF3297CEE2CA90F834EA9B2
:100860000E53C77B88215D8D6244DECD9AEF69937C
:10087000163EAC7FF2575DD06C8509CAB2A93474BC
:100880004B9D7176CD9259FD08373D09524A1A2A7F
:10089000E407A39035E7F42623EA01C0E27C438D08
:1008A000A99D6FDA84655859FAD5258C68A26392A0
:1008B000A9C43B9037A4DAA2BF73EAE5F384909F02
:1008C000A5BE34DA480861329ABE08E9599AFD1487
:1008D000048EE809001EB1579821EFF0AB97D1DFE5
:1008E000271FE5CD0015616AFCD629A0E50001C4EB
:1008F00004D11000003353623EB1C467FB02000014
:10090000000004595A504F52514A4D4B4E2A4C2F19
:1009100030B6B7ABACBBBCA9AABDBE0D0E0B0F1A4F
:100920000508050905071811130408120C00112405
:100930001FBECFEFDAE0DEBFCDBF04B603FE18C0A6
:100940008091240590912505A0912605B091270559
:100950008730904BA740B04B59F410922405109269
:1009600025051092260510922705E0E0F8E3099589
:1009700011E0A0E0B1E0EEE1F6E602C005900D92D4
:10098000AC3CB107D9F725E0ACECB1E001C01D9259
:10099000A432B207E1F70E94F2280C94A53230CBC2
:1009A0009C01FB019A9581159F4120F5832F817051
:1009B000B32FB270AA27732F74706627532F587005
:1009C000442734FF0DC08295807FAB2B09F08062F5
:1009D000672B09F08064452B09F08068099508951C
:1009E000AB2B09F08260672B09F08460452BB1F3D3
:1009F0008860F4CF80E0F2CF0C9491310895982F65
:100A000092959F7024E0911102C020E0982F892FC9
:100A100086958695811511F02E5F982F892F8695E2
:100A2000820F089581FD02C05C9A08955C98089534
:100A300080932005089580932105089521E030E0FA
:100A400001C0220F8A95EAF780912105822BF3CF0E
:100A500021E030E0A90102C0440F551F8A95E2F75A
:100A6000CA018095909121058923E5CF292F9530E2
:100A700090F58E3080F590E03EE0239F800D911D33
:100A80001124282F277041E001C0440F2A95EAF76E
:100A900023E0969587952A95E1F7FC01EE0FFF1F5D
:100AA000E80FF91FE25BFC4F20E030E070E051916D
:100AB000DF01CB01022E02C0969587950A94E2F7DA
:100AC000817081958527842385278E932F5F3F4FE3
:100AD0002330310561F70895292F953078F58E3050
:100AE00068F590E03EE0239F800D911D1124682F52
:100AF000677023E0969587952A95E1F7FC01EE0F44
:100B0000FF1FE80FF91FE25BFC4F40E050E080E080
:100B1000219130E0062E02C0369527950A94E2F71F
:100B200021703327042E01C0220F0A94EAF7822B8A
:100B30004F5F5F4F4330510559F7089580E00895A6
:100B40009091210521E030E0F90101C0EE0F8A9576
:100B5000EAF7D90102C0AA0FBB1F6A95E2F7EA2B98
:100B600001C0220F4A95EAF7892F8E23E81303C0AC
:100B7000892F822B60CF2095822F8923FBCF8091F4
:100B8000FC029091FB02981301C008958F5F87705B
:100B9000FACF90916C048095892380936C04282F60
:100BA0002770211110C0891771F09091230592FFD1
:100BB0000AC08695869586954BDF10926C0410923C
:100BC0006E0410926D04089590916904982B90938F
:100BD00069040895982F90958091690489238093E2
:100BE0006904089580916804811531F010926804B9
:100BF0001092700410926F040895803E9105D9F10F
:100C0000C8F48133910509F482C048F48932910512
:100C100009F472C08A32910509F480C008958933BD
:100C20009105E9F082389105D1F08533910509F4F9
:100C30005EC00895843E9105D9F148F4823E910545
:100C400039F1833E910549F181EE90E00895863EA9
:100C50009105C9F1873E910509F43EC008952091A0
:100C600022052370211164C02091230523FF14C0A5
:100C700089E290E008952091220520FD45C0309141
:100C8000230530FF09C024FD24C083EE90E00895C1
:100C90002091220522FDF7CF08952091220522FD03
:100CA00044C03091230530FD43C024FFF5CF11C06F
:100CB0002091230521FFF0CF8091220584FD09C0FA
:100CC00087EE90E008952091220523FFE5CF24FFD1
:100CD000F7CF80E090E008952091220523FD2BC0FE
:100CE0003091230531FFE1CF84EE90E0089520910B
:100CF000220525FFD1CFBCCF2091220525FD1EC0A6
:100D00002091230523FFC8CF89E390E00895209127
:100D1000220526FFC1CF8AE290E0089520912205A6
:100D200026FFBACF81E390E0089582EE90E0089527
:100D300080EE90E0089586EE90E0089585E390E0DF
:100D400008959091220592FF10C041E0282F247150
:100D5000243009F040E031E0282F2871283009F0D4
:100D600030E0431711F02CE0822793FF10C041E0E0
:100D7000282F2471243109F040E031E0282F287118
:100D8000283109F030E0431711F02CE08227309130
:100D9000230530FF10C051E0282F2171213009F0C8
:100DA00050E041E0282F2871283009F040E0541726
:100DB00011F029E0822731FF10C041E0282F217176
:100DC000213109F040E031E0282F2871283109F065
:100DD00030E0431711F029E0822794FD877E0895C3
:100DE0001F93CF93DF9309DFEC01811522E5920772
:100DF00008F052C0811540E5940708F0CDC0803E50
:100E0000910520F58D3C910508F0A1C0883A910527
:100E100070F4853A910508F097C081309105B9F1D9
:100E20000497813A910598F1C0E0D0E030C0885A2B
:100E300091094B97C8F7C85AD0E0CC0FDD1FC05AB4
:100E4000DE4F0990D881C02DD46421C0811550E4B3
:100E50009507B0F4C11580E2D80708F0B3C0C83ECA
:100E6000D105A8F0CE019A9581159F41E8F68D2F06
:100E700068DF182FCE019927C0DEEC01D12B07C007
:100E80009927BBDECC27DF70C82BD92BD06ACE01C7
:100E9000DF91CF911F910895803842E59407C8F5FE
:100EA000803652E5950708F05BC0C03482E5D8076C
:100EB000D0F4C03292E5D90708F04BC08C2F86954C
:100EC000869520E2829FC0011124C37021E030E0AA
:100ED000A90102C0440F551FCA95E2F7EA01C82BC9
:100EE000D92BDD68D4CF8C2F86958695877050E2FC
:100EF000859FC0011124C37021E030E0A90102C028
:100F0000440F551FCA95E2F7EA01C82BD92BDC68BC
:100F1000BECF803C52E5950758F48F71C03AD24558
:100F2000A0F590E0982F8827EC01C46FD06AAFCF6E
:100F3000805C9245809708F077CFDC2FCC27CC27B8
:100F4000DF71C06FD06AA3CFA497D064A0CFD06563
:100F50009ECFCF71D0E0DC2FCC27C16FD06A97CF66
:100F600086958695877020E2829FC0011124C37008
:100F700021E030E0A90102C0440F551FCA95E2F7F5
:100F8000EA01C82BD92BDA6882CFDBDEC82FD0E08C
:100F9000DC2FCC27D0627BCF8F71D3DE93E0CC0FD8
:100FA000DD1F9A95E1F7CC27DF70282F30E084FF12
:100FB00005C050E1859F900111243327C22BD32B0C
:100FC000D06965CF8D2F8F71BCDE182FCE01992788
:100FD00014DEEC01D12BDECF80E00895F894E82FE9
:100FE000E295EF70F0E041A18F7021E030E0B901AF
:100FF00002C0660F771F8A95E2F7CB01962F909576
:10100000942391A392A1892B82A3789408950895A3
:10101000CF92DF92EF92FF921F93CF93DF93172F20
:10102000E82FF0E0ED56FA4F71110CC0E4918E2FCD
:101030007E2F6E2FDF91CF911F91FF90EF90DF9069
:10104000CF900895E62EF12CC72ED12CF491EF2FDE
:1010500086E0689F90011124CFEFD0E0C901BE0166
:101060000E947731AB01EE0CFF1C65E5649FC00167
:10107000659F900D1124E81AF90A6E2D660F6E0D0A
:101080007E01EC18FD08FE9DD001FF9DB00D1124DE
:101090008B2F169F70011124EF2CFF246E01CE18A8
:1010A000DF087601FE9D6001FF9DD00C11247E01BA
:1010B000E61AF108B701169F7001179FF00C112472
:1010C000EF2CFF24CE19DF09FC9F7001FD9FF00C6F
:1010D00011247F2D43305105C1F02C3F334058F48B
:1010E00041305105B1F04230510509F0A2CFEB2F4C
:1010F0008F2D7F2F9ECF4430510571F04630510522
:1011000009F497CF7B2F8D2D94CF7D2DEB2F8F2F33
:1011100090CF7F2FED2D8DCFEF2D7B2FF8CFCF935D
:10112000982F762F842FC22F692F72DF472F282FF9
:101130008C2F90E0FBD0CF91089580915F04843094
:1011400028F48370846080935F0408958436E8F304
:1011500083708066F8CFCF93DF9380915F0480FD2A
:101160000BC0C0E0D0E020E040E060E0CE01DED087
:101170002196CE30D105B9F72ED4DF91CF910895C5
:10118000FF920F931F93CF93DF93182F062FF42E08
:1011900080915F0480FF0CC0C0E0D0E02F2D402F75
:1011A000612FCE01C3D02196CE30D105B9F7D3DF60
:1011B000CDB7DEB7E5E00C94D131982F762F842F90
:1011C00020915F0420FF07C0692F22DF962F672F31
:1011D000482F892FD5CF0895CF93DF93EC01EFE50A
:1011E000F4E0438162818C81E8DF8C818F5F8C83A6
:1011F000DF91CF910895CF93DF93EC01EC81F0E084
:10120000E257FB4F4491EFE5F4E062818181D5DF45
:101210008C818F5F8C83DF91CF910895FF920F9324
:101220001F93CF93DF93EC01F12C00E010E08C8151
:10123000980140916204609161048F0D70DF0F5F2F
:101240001F4F82E1F80E0E30110589F784DF8C8183
:101250009A8190FF07C08F5F8C83CDB7DEB7E5E042
:101260000C94D1318150F8CF81152CE7920741F4CD
:101270002091C8023091C902232B11F480E090E044
:101280000895E7EDF3E080E090E06EEB76E241EE6A
:1012900056E223E537E277836683518740873387B9
:1012A000228797878687019670968830910599F7EF
:1012B0000895FB01811520E2920728F4811541E091
:1012C000940738F408959C0130522115304348F0BA
:1012D0000895392F94FF02C03295307F2081232B4F
:1012E000208399270895462B22FF0FC0982F9295AF
:1012F0009F708F70892B962F92959F706F70692BBE
:10130000942F92959F704F70492B982F9623961388
:1013100009C050E04095509590E04823592381E062
:10132000452B09F080E00895869A0895FC01EE0FA0
:10133000FF1FE80FF91FE95EFD4F618340832283A1
:1013400008951092B2041092B104E1E7F4E08581AF
:10135000811102C014821682379684E0E93AF807B8
:10136000B1F70895AC013091B4046091B304232F18
:10137000621301C00895822F90E0FC01EE0FFF1F61
:10138000E755FB4F0190F081E02DE417F50791F44C
:1013900067E0649FF001659FF00D1124EF58FB4F4B
:1013A00041E044832313E6CF01968370992780930D
:1013B000B40408950196282F2370DACF0F931F935A
:1013C000CF9301E010E0082E01C0000F0A94EAF765
:1013D000C09167049C2F9023911115C090916C04CB
:1013E000969596959695891306C010926C04109266
:1013F0006E0410926D0422DBC027C0936704CF9166
:101400001F910F91089524DBF7CF9091BE038902BD
:101410009001112437FF03C08093BE0308952F3736
:1014200031051CF4980F9093BE0308959C0180E051
:1014300090E0F901E80FF91FE491E41307C091E08F
:101440008927F901E80FF11D849108950196861707
:1014500080F380E00895FA01309709F00995089526
:10146000E091F102F091F202309739F00190F081B1
:10147000E02D309711F00995089580E00895A3E0DC
:10148000B0E0E5E4FAE00C94B8319C0180911402DC
:101490009091150282179307B1F0309315022093B3
:1014A0001402E091F102F091F202309761F00084B1
:1014B000F185E02D309739F083E089833B832A83DF
:1014C000CE01019609952396E2E00C94D431A3E075
:1014D000B0E0EDE6FAE00C94B8319C018091120284
:1014E0009091130282179307B1F030931302209367
:1014F0001202E091F102F091F202309761F0008463
:10150000F185E02D309739F084E089833B832A838D
:10151000CE01019609952396E2E00C94D431909186
:101520001901913091F0A0EDB1E0EFEF90E02D9135
:10153000821751F0EF3F19F4211101C0E92F9F5F8D
:101540009630A9F7EF3FC9F408959091220597FFCF
:10155000EACFE82FE695E695E695803FA8F7F0E01C
:10156000EA52FE4F877021E030E001C0220F8A95D9
:10157000EAF78281822B828308950E2E000CFF0BE6
:10158000E253FE4FF8CF90911901913021F49091E0
:10159000220597FD0CC0E0EDF1E09191891302C0A6
:1015A000DF011E9251E0E63DF507B9F70895E82FF7
:1015B000E695E695E695803FC8F7F0E0EA52FE4FE3
:1015C000877021E030E0A90102C0440F551F8A95C1
:1015D000E2F7CA01809592818923828308958091E0
:1015E000180108952FB7F89480910E0290910F0280
:1015F000A0911002B09111022FBF0895CF93DF93F5
:10160000C091690480916B04C82B80916804811596
:10161000F1F0E8DF20916F0430917004821B930B8E
:101620008838934108F0DEDAD0916804809119017E
:10163000813021F48091220587FD0DC086E020EDE8
:1016400031E090E0815058F49111CCDACD2B8C2F01
:10165000DF91CF9108958EE128ED31E0F2CFF901CD
:1016600041919F01411571F39F5FECCF962F20911F
:10167000230522FF0EC0682F660F660F660F692BC9
:1016800060936C04DBD9AEDF90936E0480936D049D
:101690000895D4C990916804292F2823211559F061
:1016A0008095892380936804811531F09BDF8093B6
:1016B0006F0490937004089580E090E0F8CF2FB706
:1016C000F89460910E0270910F0280911002909137
:1016D00011022FBF08950895FC019B01809104021F
:1016E000909105028617970740F0672B29F48091A7
:1016F000E8008E778093E800C90140E0009741F44C
:10170000411106C08091E80082FF2FC080E008955B
:101710002091CA022115A9F12530A9F12091E800F4
:1017200023FD2DC02091E80022FDECCF2091E800A0
:1017300020FFE4CF3091F3002091F200009719F0E0
:101740002830310558F041E02830310509F040E0FB
:101750002091E8002E772093E800D0CF419140936C
:10176000F10001972F5F3F4FE9CF8091CA028115A9
:1017700041F0853041F08091E80083FFC3CF81E0E4
:10178000089582E0089583E008958091FE0187FF27
:1017900013C08091E80082FF06C08091E8008B773B
:1017A0008093E80008958091CA028111F2CF0895D4
:1017B0008091CA028115D9F38091E80080FFF8CFAB
:1017C0008091E8008E77ECCF2091E4003091E50025
:1017D00095E6A9012091EC00822F817020FF06C0C0
:1017E0008091E80080FF06C080E008952091E80025
:1017F00022FD1AC08091CA02811589F0853089F0D6
:101800008091EB0085FD0FC02091E4003091E50050
:1018100042175307F9F29A95E1F684E0089582E0C1
:10182000089583E0089581E00895E8EDF0E0808177
:101830008E7F80831092E2001092DA001092E10015
:10184000A0EEB0E08C9181608C9380818F77808353
:1018500019BCA7EDB0E08C918E7F8C9380818F7E38
:1018600080831092FD010895E091F102F091F2025F
:10187000309739F00284F385E02D309711F060E263
:1018800009950895982F9093E900891771F0709148
:10189000EC002091ED005091F00021FD09C09F5F08
:1018A000973089F78093E9000895762F242F50E030
:1018B0003091EB003E7F3093EB003091ED003D7FA7
:1018C0003093ED003091EB0031603093EB0070937A
:1018D000EC002093ED005093F0002091EE0027FDE6
:1018E000DECF0895A0E0B0E0E8E7FCE00C94B23170
:1018F000C8EDD0E088818F7E8883E7EDF0E08081BD
:101900008160808384E082BF81E08093FD018881D3
:101910008E7F888302EE10E0F80110821092DA00C8
:1019200081EEC82ED12CF601108288818F778883B2
:1019300088818068888388818F7D888319BC109214
:10194000CA021092FC011092A7021092FB0190EEC5
:10195000E92EF12CF70180818B7F80838881816063
:10196000888342E060E080E08DDFF60180818E7F39
:101970008083F8018081816080838081886080839A
:10198000F70180818E7F8083888180618883CDB7D5
:10199000DEB7E8E00C94CE31E091FC029091FB02BE
:1019A00029E0E91302C080E00895AE2FB0E02E9F39
:1019B000F0011124E350FD4F3181361306C0308110
:1019C000381303C03581341304C0FD013196E7702C
:1019D000E8CF81E0089531B33F7B21B320644FB756
:1019E000F89487E192E0FC010196508168E021BB08
:1019F000000000C057FF31BB550F000000C000C001
:101A000000C031BB00C06A9591F752E08134950760
:101A100051F74FBF8FE594E00197F1F700C0000048
:101A2000089581E08093E00080E28093D8001092D6
:101A3000C9008FE19EE40197F1F700C0000087E044
:101A400090EBDC018093240590932505A093260557
:101A5000B093270588E19CE00FB6F894A895809391
:101A600060000FBE90936000FFCF0F931F93CF9342
:101A7000DF938B01EA019091CA02943051F5809373
:101A8000E9008FEF9091E80095FD06C095ED9A95DD
:101A9000F1F700008A95B1F78091E80085FF19C041
:101AA00093DE811111C08091E80085FD06C0809110
:101AB000E8008E778093E800F3CFF80181918F01E1
:101AC0008093F100219779F78091E8008E778093D9
:101AD000E800DF91CF911F910F910895792F603227
:101AE00029F440E250E0682F82E0BFCF0895CF9301
:101AF000DF93D82FC92F48E050E0682F792F81E07D
:101B0000B4DF88E0ED2FFC2FA6E0B2E001900D924B
:101B10008A95E1F7DF91CF910895BC0140E250E052
:101B200084E0A3CFBC0143E050E084E09ECF9091DD
:101B3000230592FB222720F9281771F080FB92F9E8
:101B400090932305609122057091230584E090E035
:101B50000E948A3282E01DC808951F93CF93DF93BD
:101B6000962F122F632F8430D8F49530C8F44E305E
:101B7000B8F4C42FD0E0CC0FDD1F2CE1929FC00D34
:101B8000D11D11249CE8899FC00DD11D1124CE01C7
:101B900089960E947032612FCE018A960E9470321F
:101BA000DF91CF911F91089580911901813061F5E6
:101BB0008091220587FF28C021DD8093D70140E274
:101BC00050E061ED72E086ED91E00E942B32892BAE
:101BD000D1F080E2E6EDF1E0A1EDB2E001900D92EE
:101BE0008A95E1F7E091F102F091F202309759F015
:101BF0000480F581E02D309731F086E08093D601A6
:101C000086ED91E009950895F9DC8093CE0148E0D6
:101C100050E063EF72E08EEC91E00E942B32892B52
:101C200091F388E0EEECF1E0A3EFB2E001900D92C9
:101C30008A95E1F7E091F102F091F202309719F301
:101C40000280F381E02D3097F1F28EEC91E0DACF53
:101C5000CF93C82F8115A1F08238A1F401DC81FD5A
:101C60000FC089E35CDCA0DF2FEF37EE83E021506B
:101C700030408040E1F700C0000089E384DC94DF5D
:101C8000CF910895833889F4EBDB80FDF9CF83E5AC
:101C900046DC8ADF9FEF21EE34E091502040304057
:101CA000E1F700C0000083E5E9CF843889F4D8DB90
:101CB00082FDE6CF87E433DC77DF8FEF91EE24E01F
:101CC000815090402040E1F700C0000087E4D6CF6B
:101CD0008CEF8C0F813A78F580911901813069F091
:101CE000E0EDF1E086ED91E02191C21701F18E1750
:101CF0009F07D1F78C2F13DCC2CF8091220587FF7D
:101D0000EFCFEC2FE695E695E695F0E0EA52FE4F30
:101D1000828190E04C2F477021E030E002C0220F1A
:101D2000331F4A95E2F782239323892B19F38C2FD3
:101D30002ADC3ADFDFCF80E28C0F883048F4C770AE
:101D400081E001C0880FCA95EAF70E94E40597CFA9
:101D50008BE58C0F833030F42C2F2452330BC901C8
:101D60008EDB8ECFC85ACB3108F08ACFEC2FF0E053
:101D7000EE0FFF1FEA56FE4F80819181A8DB80CFD6
:101D8000811509F43EC0823849F46ADB81FF39C00D
:101D900089E3C5DB09DF89E3F6DB06CF833841F44D
:101DA0005FDB80FF2EC083E5BADBFEDE83E5F4CF88
:101DB000843841F455DB82FF24C087E4B0DBF4DED5
:101DC00087E4EACF9CEF980F913A30F390E2980FB6
:101DD000983050F4877091E001C0990F8A95EAF726
:101DE000892F0E94EA05D9CF9BE5980F933018F40C
:101DF00080E090E044CB885A8B3118F480E090E08A
:101E000066CB08951F93CF93DF93182FEB0120DF4C
:101E1000209731F4812FB4DFDF91CF911F91089586
:101E20008FE99FE00197F1F700C000002197F0CF04
:101E3000811519F00E94E405B7CE0895811519F0B7
:101E40000E94EA05B1CE0895811531F090916B049E
:101E5000892B80936B04A8CE0895811539F0809565
:101E600090916B04892380936B049ECE089580919A
:101E7000D303811521F082E2F0DF1092D30308959D
:101E800010926904809119018130A1F4809122059A
:101E900087FF10C0E8EDF1E08EE1DF011D928A9529
:101EA000E9F780E090E0EBDA80E090E010DB109260
:101EB0006B047ACEE0EDF1E086E0EFCFE1DF2FEFCB
:101EC00084E39CE0215080409040E1F700C0000096
:101ED00088E19CE00FB6F894A895809360000FBE4F
:101EE00090936000FFCFAAE2B0E0E9E7FFE00C9436
:101EF000B7318EEF91E0FC0101962091F100208333
:101F000022E086309207B9F78091FF01893009F409
:101F100057C0C8F4823009F4B2C0833009F482C0DB
:101F2000813081F18091E80083FFE6C08091FE015D
:101F30009091FF019A3008F0DFC0E92FF0E0E955F9
:101F4000FD4C0C948B318A3009F489C08B3051F7E9
:101F50008091FE01813231F780910202909103025B
:101F6000892B01F78091E800877F8093E8000DDCE2
:101F700081E090910002911101C080E080931901ED
:101F80007FDFD0CF8091FE01813A61F68091E80039
:101F9000877F8093E8008091020290910302892B51
:101FA00059F060E080E090E070E096DB8091E8001E
:101FB0008B778093E800B6CF68E086E092E0F4CFBC
:101FC0008091FE01813209F0ADCF809102029091A3
:101FD00003028D7F892B09F0A5CF8091E800877FD0
:101FE0008093E8008091E80082FF17C09091F30091
:101FF0008091F200029731F48091F100813011F06C
:10200000863021F48091F100809318018091E800DE
:102010008B778093E800B9DB85CF8091CA0281116C
:10202000E1CF80CF8091FE01813A09F07BCF809192
:10203000020290910302892B09F074CF8091E8008D
:10204000877F8093E8008091E80080FFFCCF80913B
:1020500019018093F1008091E8008E77DACF8091AA
:10206000FE01813209F05ECF8091E800877F809386
:10207000E8008BDB809101028093170153CF8091A0
:10208000FE01813A09F04ECF8091E800877F80936E
:10209000E8008091E80080FFFCCF80911701D9CF44
:1020A000803889F0823841F5809102028F70873044
:1020B00018F58093E9008091EB0085FB882780F973
:1020C0001092E90006C08091A702880F9091FB0151
:1020D000892B9091E800977F9093E8008093F1001E
:1020E0001092F1008091E8008E7723C0811116C014
:1020F00080910002813009F18091E80083FF0AC0DD
:102100008091E800877F8093E8008091EB008062F7
:102110008093EB00AA96E3E00C94D331823061F710
:1021200080910002811581F01092E9008091E80011
:10213000877F8093E80029DBDFCF81E0933009F0CF
:1021400080E08093A702F0CF809102028F702FEF82
:10215000280F263088F68093E9002091EB0020FFBD
:10216000E3CF933031F48091EB0080628093EB00F9
:10217000DBCF9091EB0090619093EB0021E030E099
:10218000A90102C0440F551F8A95E2F74093EA0067
:102190001092EA008091EB008860E8CF8111ACCF0B
:1021A000109100021F778091E3008078812B80934B
:1021B000E3008091E800877F8093E800E6DA809171
:1021C000E80080FFFCCF8091E30080688093E3000B
:1021D00083E0111101C082E08093CA028DCF805844
:1021E000823008F089CF80910002909101028C3DED
:1021F00053E0950791F583E08A838AE289834FB79C
:10220000F894DE01139620E03EE051E2E32FF0E087
:1022100050935700849120FF03C082958F703F5FD9
:102220008F708A30C0F0895C90E08D939D932F5F12
:10223000243161F74FBF8091E800877F8093E800E9
:102240006AE270E0CE01019647DA8091E8008B7770
:102250008093E80051CF805DE7CF292F33272330CB
:10226000310509F44EC078F52130310509F488C0F4
:102270008BE590E0EFE2F2E02230310509F03CCF4F
:102280002091E800277F2093E800209104023091FC
:1022900005028217930708F49C0140E021153105DF
:1022A00009F073C0411171C08091E80082FDCDCF6B
:1022B0008091CA02811549F2853039F28091E80097
:1022C00083FFF2CFC2CF80910202909103022132AC
:1022D000310509F446C02232310509F00DCF8330B3
:1022E000910508F009CFFC01EE0FFF1FE85DFE4FDE
:1022F0000190F081E02D8B5D9E4FDC018C9190E090
:1023000010C09C013327823021F12330310568F45D
:10231000232BB9F4E6EEF2E0E4918E2F90E0E6EEA6
:10232000F2E0009709F4E8CEABCF2330310509F095
:10233000E3CEECE9F2E0E4918E2F90E0ECE9F2E0FC
:10234000F0CFE2EDF2E0E4918E2F90E0E2EDF2E0EA
:10235000E8CFEAEBF2E0E4918E2F90E0EAEBF2E0D6
:10236000E0CF8330910508F0C7CEFC01EE0FFF1FD0
:10237000E25DFE4F0190F081E02D89E090E080CF9A
:1023800082E190E0EAE8F2E07BCF8091CA02811519
:1023900009F45BCF853009F458CF8091E80083FDC4
:1023A00054CF8091E80082FD7FCF8091E80080FFCC
:1023B00075CF9091F3008091F2002115310519F04D
:1023C0008830910550F041E0089709F040E0809195
:1023D000E8008E778093E80061CF44914093F1004C
:1023E0003196215031090196E8CF803809F084CE2A
:1023F0008091E800877F8093E8008091FC018093C2
:10240000F10070CE811178CE10910002123008F0E8
:1024100073CE8091E800877F8093E8001093FC01E1
:10242000B4D91115D9F084E08093CA0242E061EC7E
:1024300081E028DA42E261EC84E024DA42E261ECF5
:1024400082E020DA42E260EC83E01CDA8091CA028A
:10245000843051F482E080931A014ECE8091E300E3
:1024600087FDE1CF81E0E0CF81E0F5CFCF93DF932F
:10247000EC014A855B856E857F850E942B0A9B81D6
:10248000909580916B04892380936B048C810E94CA
:10249000EA058ADB86E0FE0111928A95E9F7DF9171
:1024A000CF910895CF93DF93EC018D8181FD13C00F
:1024B00082608D8380916B049B81892B80936B0458
:1024C0008C810E94E40570DB488559856E857F8587
:1024D000CE010E942B0A10925804109257048D814D
:1024E00080FD02C0CE01C2DFDF91CF9108950F932E
:1024F0001F93CF93DF93843030F5653020F54E3055
:1025000010F5C42FD0E0CC0FDD1F2CE1629FC00D71
:10251000D11D11243CE8839FC00DD11D1124CE0193
:1025200089960E944F32082F10E0102F0027CE010D
:102530008A960E944F329801282BC901DF91CF91D2
:102540001F910F91089580E090E0F8CF462F672FFC
:102550002091CD023091CE02232B81F4703F39F4CB
:10256000403F61F48091CB029091CC020895753088
:1025700028F44E3018F4843008F4B9CF80E090E0AD
:102580000895A0E0B0E0E7ECF2E10C94B3317C01F7
:102590000091210580912005082BC3E0D0E010E0D8
:1025A000C8010C2E02C0959587950A94E2F780FD2C
:1025B00009C02197A8F7D12C8D2DCDB7DEB7E7E064
:1025C0000C94CF31DC2EB7018C2FC0DF0E94F006B7
:1025D000019779F3F1CF0F931F93CF93FC0187817C
:1025E0009085009789F4858100811181811581F0A2
:1025F000611571F0C801C5DFC82F682FC8010E949E
:102600003605B8018C2FA2DFCF911F910F9108954D
:10261000C8010E946C05C82FF4CFCF93DF93D82F49
:10262000C92FAFDF6D2F7C2F91DF0E94F006DF9165
:10263000CF910895FC0184818115B1F08781908547
:102640000097A1F00E94F006282F92959F70963077
:10265000B9F080F4925F9F70923030F4203FD1F057
:1026600058F481E0283E58F080E0089580819181FF
:10267000D4DFEACF9A5FEFCF81E0243FA9F7089536
:1026800091E0813F09F090E081E0283E08F080E091
:10269000892B089581E00895382F292FCB01A32F8E
:1026A000B22F873D9105A105B10520F4875D9C4FB0
:1026B0000C944F3280E0089585E290E00E944F3202
:1026C000843E89F486E290E00E944F328E3259F4C3
:1026D00087E290E00E944F3291E0883909F090E063
:1026E000892F8170089580E0FCCFA0E0B0E0EBE797
:1026F000F3E10C94B131EC018881811509F181304D
:1027000009F045C08981813051F48A81239660E5C2
:1027100070E0893311F060E070E074DBEDCF82305F
:1027200021F48A81239694DAE7CF833021F48A81D9
:10273000239626DBE1CF843041F022968111DCCF55
:10274000CDB7DEB7E9E00C94CD318A81239620E045
:1027500030E09AE0682F6053770BAB016A30710567
:1027600060F02115310551F3EFE9FFE03197F1F702
:1027700000C0000021503109F4CF929FB001939F17
:10278000700D11249A01260F371F8991E3CFE82F8E
:10279000F0E0E155FE4FB490282F2695269526951A
:1027A00030E0F901E156FE4FE4908770F12C082EDD
:1027B00002C0F594E7940A94E2F7E0FAEE24FF24CD
:1027C000E0F8F901E157FE4FC490D12C082E02C069
:1027D000D594C7940A94E2F7C0FACC24DD24C0F85B
:1027E000F901E158FE4F049110E002C015950795DC
:1027F0008A95E2F701701127E114F10411F081EEDE
:1028000027DAC114D10411F086EE22DA60E070E01C
:102810008B2DF8DAC114D10411F086EEB1DAE1148F
:10282000F10411F081EEACDA0115110521F060E040
:1028300070E08CE2E7DA21965FCFAAE0B0E0E3E255
:10284000F4E10C94AD31C090C802D090C90281E08F
:1028500090E09093C9028093C802812C912C10E0E3
:10286000540100E019C021E030E0133021F0F701FD
:10287000859195919C01472D602F812F6ED973947E
:1028800022E0E20EF11C3EE07312EDCF0F5F8EE00E
:10289000A80EB11C053049F0C501880F991FFC0135
:1028A000E651FD4F7F01712CDECF1F5FF6E48F0EE6
:1028B000911C1430A9F61A8219821C821B821E8276
:1028C0001D8218861F8288EC90E09A87898709E527
:1028D00012E09E012F5F3F4F79014AE050E0B801BE
:1028E000C7010E948E32065F1F4F093A32E013077C
:1028F000A1F78AE0F70111928A95E9F74AE050E0E2
:10290000B801C7010E948E32065F1F4F093FF2E0F7
:102910001F07A1F786E0F70111928A95E9F746E0D3
:1029200050E0B801C7010E948E320A5F1F4F093282
:10293000F3E01F07A1F7D092C902C092C8022A96FD
:10294000EDE00C94C931AAE0B0E0E9EAF4E10C94BE
:10295000B231E1E4F2E080E5DF011D928A95E9F70A
:10296000E1E7F4E088E3DF011D928A95E9F781E46D
:10297000C82E82E0D82E7F0109EA12E0F701D18249
:10298000C0824AE050E0B801CE0101960E943F3279
:1029900088E0FE013196D60101900D928A95E1F70B
:1029A00089859A85D70113969C938E931297BAE0E6
:1029B000CB0ED11CE7E0EE0EF11C065F1F4F093F66
:1029C000F2E01F07D9F62A96E8E00C94CE31A6E093
:1029D000B0E0EDEEF4E10C94B33103E713E089EFDE
:1029E000E82E82E0F82E98E0D92E46E050E0B701BC
:1029F000CE0101960E943F32F8018D2D11928A95E9
:102A0000E9F7B8016C5F7F4F89819A810E9459096B
:102A1000F80191838083B8016B5F7F4F8B819C812C
:102A20000E945909F801938382838D8186838E8168
:102A30008783F6E0EF0EF11C085F1F4F89E2E8166E
:102A400083E0F80691F62696E7E00C94CF31282F24
:102A5000CB01283070F44AE0249F90011124B90181
:102A6000675A7D4F4AE050E00E943F3280E090E09C
:102A700008958FEF9FEF0895AAE0B0E0E2E4F5E15A
:102A80000C94B8319C0197558115914068F4BE01B2
:102A90006F5F7F4F822FDBDF892B31F489859A8529
:102AA0002A96E2E00C94D43188EC90E0F9CFA0E0D3
:102AB000B0E0EDE5F5E10C94B331162FD72FC42F1C
:102AC000D22E8115A1F040935B040E94F20A9093EC
:102AD000FA018093F901C77081E001C0880FCA959F
:102AE000EAF7A6D9CDB7DEB7E7E00C94CF319091E5
:102AF0005B04491335C0E090F901F090FA010E949F
:102B0000F20A9C012E193F097901812F9D2FB4DF14
:102B1000E816F90628F5D0E2DD0DCD1591F0C77065
:102B200011E0812F01C0880FCA95EAF787D9D83004
:102B300040F48D2D877001C0110F8A95EAF7812F1F
:102B400077D960E070E0802F5DD9D83058F62D2D10
:102B5000277081E001C0880F2A95EAF76FD9C2CFAC
:102B6000C77081E001C0880FCA95EAF7F7CF0F93CD
:102B7000CF93DF93CFE5D4E0488159816A817B818F
:102B800088E090E00E948232288139814A815B810D
:102B90006C817D818E819F8100E20E94FA31622FDB
:102BA00083E290E00E947032DF91CF910F910895FF
:102BB000EFE5F4E085E0808311828FEF82838383E9
:102BC0001482CF01D4CF80916304833018F48F5FD7
:102BD000809363048FE594E0CACF809163048115EC
:102BE00019F08150809363048FE594E0C0CFA0E09A
:102BF000B0E0EDEFF5E10C94AD31182FF62E042F77
:102C0000E22E90915F0490FF23C0E92FE695E695B0
:102C1000AE2FB0E0AC5CBE4F8C9180935D049C7F86
:102C20009430D9F4612F7F2D842F0E940808962FAD
:102C3000672F482F892F0E94C00810936004F092DC
:102C4000610400936204E11419F08FE594E08FDFD2
:102C5000CDB7DEB7EDE00C94C931823019F40091A4
:102C60006204EBCF863019F410916004E6CF89300E
:102C7000D9F38F3011F7EF508E2F8170782EE695B3
:102C8000F0E0E257FA4FE491CE2FD0E0A12CB12C26
:102C9000C12CD12C8EE0882E912CC501B4010E944C
:102CA0007731812F711012C0860F9601402F6F2D42
:102CB0000E948F088FEFC81AD80AAC0EBD1E8EE096
:102CC000C816D10451F70E94AB08B7CF861BEDCFD1
:102CD000EFE5F4E0818121E043816281885F87CF65
:102CE000EFE5F4E0818121E04381628188507FCF6C
:102CF000EFE5F4E0628128E0620F08F46FEF21E075
:102D00004381818174CFEFE5F4E0628128E0621BAA
:102D100008F460E021E04381818169CFEFE5F4E0D0
:102D2000438128E0420F08F44FEF21E06281818166
:102D30005ECFEFE5F4E0438128E0421B08F440E079
:102D400021E06281818153CF60915F046695669531
:102D500070E04BE050E080E091E00E941E32892B51
:102D600019F481E080935E040E94F20A9093B40209
:102D70008093B302089590915F0490FF2CC0811559
:102D800059F1893158F58F73880F880F90915F043E
:102D90009370892B80935F04611519F08FE594E09F
:102DA000E6DE60915F046695669570E04BE050E06A
:102DB00080E091E00E941E32892B91F010925E0417
:102DC00081E08093B60220E040916204609161044A
:102DD000809160040CCF089581E0D6CF88E1D4CFF4
:102DE000B3DFEECF80915F04869586958F5F893142
:102DF00008F081E061E0BFCF80915F048695869501
:102E00008A9509F488E161E0B6CFAAE0B0E0EBE092
:102E1000F7E10C94A8317C01DC0114968C918115AA
:102E200009F449C161E0C701D6DB8C01F701858156
:102E3000811521F180915704909158040097F1F089
:102E400008171907D9F0FC01FF27887F9927892BDC
:102E500009F04BC0A4E0EE0FFF1FAA95E1F7E9527D
:102E6000FC4F85818460858311830083CF011ADB49
:102E700010926B0461E0C701AEDB8C018091C80346
:102E800081113AC0D70115968C91811509F4C9C0FA
:102E90000115B0E51B0708F0AFC00115E0E21E0701
:102EA00008F00DC10115F7E01F0731F108F5C80161
:102EB000805E9109089700F13091690480916B045C
:102EC0002091680499E0F701A4EBB3E001900D9222
:102ED0009A95E1F71093BC030093BB031092BE03D5
:102EE000832B822B8093B30307C0E0E0F0E0B9CFDF
:102EF00001153FE0130701F7D70115968C91811159
:102F0000DBC10115A7E51A0708F4E5C20115B8E50C
:102F10001B0710F00C947C206801E7E5DE1A69ECD1
:102F200073E08C2D94DD892B31F5C60174E0880F98
:102F3000991F7A95E1F7FC01E952FC4F228121307B
:102F400009F09AC22091C9033091CA03232B99F04A
:102F50002091CB033091CC03232B69F02091CD033A
:102F60003091CE034091CF035091D003242B352BC9
:102F7000232B09F48BC28091D303811509F494C3E8
:102F8000C0906904D09068040E94F20A88579C4E51
:102F90009093D5038093D403F7018581811509F4BB
:102FA00083C38D2D8C298D7981114FC30115F0E5D7
:102FB0001F0708F0E7C2011520E4120708F05DC3FF
:102FC000063E110509F40CC3C801905281159042C8
:102FD00008F05AC3D70116968C91803108F42DC39E
:102FE000C801992710926B048D32910509F0E3C254
:102FF00082E080936B044CC3003E42E5140750F41A
:10300000003652E5150708F077CFC8019255803495
:10301000910551CF980127573C472530310508F0DD
:103020004BCF0937BCE71B0709F04EC02091BB030B
:103030003091BC03232B79F18115A1F081E00E942E
:10304000050A8091B3030E94240F89E0E4EBF3E0CA
:10305000AAE6B3E001900D928A95E1F78091BE0354
:103060008093690386E0F701AAE6B3E001900D9230
:103070008A95E1F7809169038093C8038AE693E01B
:10308000C4DE1092C803F7018581811104C08091CC
:10309000B3030E942D0F80916C048770811559F045
:1030A000F7018581811539F08091230582FF03C0E6
:1030B00082E00E94C9052A96E2E10C94C431D7014E
:1030C00016968C918031F7CE0A37FCE71F0709F07E
:1030D00013CF811509F4C5C0A090BB03B090BC0309
:1030E0002091B3032D832983BE016F5F7F4FC501FC
:1030F0000E9459092C0139813A87F3E7CF2EF3E07A
:10310000DF2E01E010E022242A94D60117963C908D
:10311000179733FE53C06D907C90119712968D9047
:103120009C90139746145704B9F41496BC91B98730
:10313000232DF60146816B2F8A850E947309811524
:1031400059F089850E94FC04281634F4D60115969E
:103150009C918401192B282E84149504C9F431FE06
:1031600017C0F601F581F987232DD60116964C91EB
:103170006F2F8A850E947309811551F089850E94FD
:10318000FC0428162CF4F60194818301192B282EB7
:1031900030FE14C0FFEF2F1211C00130110571F481
:1031A000232DD60116964C9160E08A850E94730902
:1031B000811521F0F60185818401182BF8E0CF0EEE
:1031C000D11C23EB33E02C153D0509F09ECF0130D7
:1031D0001105E1F58D8182958F703D81832B8F7074
:1031E00011E0303108F410E01295107F182BA11473
:1031F00040E2B40620F5A11451E0B50608F055C030
:103200000A2D812F8D704A2D811509F451C06AE075
:1032100083E299E00E94160A282F30E0211531053B
:1032200051F4402F66E185E099E00E94160A282FAC
:1032300030E0811549F0F901F12B8F0107C0C5017C
:1032400090528115904390F100E010E087E0EFEBA1
:10325000F3E0DF011D928A95E9F71093C70300930D
:10326000C6038091C6039091C703892B09F413CF3D
:10327000F7018581811539F08FEF0E94050A809151
:10328000BE038093BD0386E0F701AFEBB3E001908E
:103290000D928A95E1F78091BD038093C8038FEB6F
:1032A00093E0B3DD1092C803F6CE1B29BB24A8CF50
:1032B00068E08BE199E0AECFC8019757803891055F
:1032C00008F0EEC0003108F0E6CE66ED70E080E078
:1032D00090E0E2D98111DFCE812C912C54010111B3
:1032E00043C004E0AE014F5F5F4F6A01D601E02F9B
:1032F0001D92EA95E9F724013501FFEF4F1A5F0AA5
:103300006F0A7F0AC501B401C7D98983811509F401
:10331000C2CE813009F0ADC0A50194012E5F3F4FB0
:103320004F4F5F4F2D833E834F835887C301B201B8
:10333000B3D9182F8A83811509F4ADCE8FEF810F91
:10334000833060F56D817E818F819885A5D98B83CF
:10335000811511F0C601C9D92401350133E0430EAE
:10336000511C611C711C17C0F7ED8F169104A1044C
:10337000B10409F490CEC501B4018ED92FEF821AA1
:10338000920AA20AB20A8111EFCF0150A8CF4D8054
:103390005E806F80788453014201A8CF8BEF810F4C
:1033A000833090F52401350143E0440E511C611C2B
:1033B000711C6D817E818F8198856ED98B8381157B
:1033C00051F3C301B20168D98C83811108C0240173
:1033D000350154E0450E511C611C711CDCCF8B8102
:1033E0009C818130AFEF9A0710F0982F8827163014
:1033F00029F0173031F00E94B326E9CF0E944F2602
:10340000E6CF0E948126E3CF143009F0C0CF6D8152
:103410007E818F81988540D9182F24013501B4E031
:103420004B0E511C611C711CC501B4016D5F7F4FB7
:103430008F4F9F4F31D9111509F42DCE811509F405
:103440002ACE8150990B4FEF489F9001499F300D34
:103450001124E12FE150FF0B2E0F3F1F21503109A6
:1034600008F499CF8FE99FE00197F1F700C00000C1
:10347000F5CFC6013AD98FCF223009F07CCD20910B
:10348000CD033091CE03232B09F475CDFC01E4521A
:10349000FC4F20812E7F208389529C4F03D86BCD17
:1034A0000337FCE71F07B9F48091D303811519F0A6
:1034B0000E94370FF0CD109269040E94F2050E941D
:1034C000F20A88579C4E9093D5038093D40381E0F1
:1034D0008093D303E0CD023A22E51207C1F158F4FC
:1034E000C80190528115904218F1013E110579F101
:1034F000053E110503C0023B52E5150709F03BCD1F
:1035000025EE30E02770332781E090E001C0880F7E
:103510002A95EAF72091D6033091D3033115F9F0BB
:10352000F70135813115B1F0282B2093D603B3CDA7
:10353000D70116968C91803108F01DCD812F9927E7
:103540008F7199278230910511F04297D7CF21EEE4
:1035500030E0D8CF809582238093D6039CCD322F44
:103560003823311509F407CD982F90959223909325
:10357000D6030E94EA05D70115968C91811509F4AE
:103580008ACDF9CC003EB2E51B0708F049C0003CEB
:10359000E2E51E0728F5003AF2E51F07E8F40036D9
:1035A00022E51207E8F4C801925580349105C0F075
:1035B00010926B04C8018E32910508F0BCC08832AD
:1035C000910508F063C08E31910508F061C0049741
:1035D0004A9708F40DCD39C0043B32E5130741F793
:1035E000F7019581911509F4A3C510925B04980128
:1035F00030572332310508F083C584E090E00E9403
:103600005C329093230580932205F801E150F04746
:10361000E232F10508F0E3C0EF54FD4C0C948B311D
:1036200009374CE7140728F407375CE71507C0F69D
:10363000BFCF0B378CE71807D2CF812F8F71843122
:1036400079F2863149F410926B040E94370F809111
:10365000D6030E94E40528C00E94370F8091D6034C
:103660000E94E405F801E851FC47E730F10508F055
:10367000B7CFED52FD4C0C948B31D70116968C913F
:10368000803108F0ADCCEECFC801ACCC8A97E9F61A
:103690008091D603811531F080916B0492E08927E7
:1036A00080936B040E94D40DC801975581159140F9
:1036B000C8F65801F8EFAF22BB24A114B10409F0F9
:1036C000EACCF801FF2754E0EE0FFF1F5A95E1F70F
:1036D0009F0129523C4F6901D70115968C91E45204
:1036E000FC4F908180FB90F99083811559F10E94E5
:1036F000F20A90935A0480935904F60182818F5FF5
:10370000828380916B0490916904892B83838091DB
:10371000680484834681578166857785C6010E9447
:103720002B0AD60115968C9181FF5801B09258044E
:10373000A092570455CF8C34910509F4A9CF8D324E
:103740009240A5CFF9014485558566857785C901E5
:103750000E942B0AD60115968C9181FF41CFC6019C
:103760000E94361280915704909158040817190747
:1037700009F036CF109258041092570431CF06E268
:1037800021EE41EE6AE17CE7F701858108C007E29E
:1037900025EE45EE6BE17CE7D70115968C9187D934
:1037A0007ACC06E221EE40EE68E17CE7EDCF07E25D
:1037B00025EE44EE69E17CE7EFCF06E221EE42EE32
:1037C0006CE17CE7E1CF07E225EE46EE6DE17CE7B8
:1037D000E3CF08E221E045EE6EE17CE7D5CF8091B2
:1037E0002205816080932205609122057091230556
:1037F00084E090E00E948A320E94400F4CCC80917D
:103800002305886080932305EFCF80912205826095
:10381000E9CF809122058460E5CF80912205886000
:10382000E1CF809123058160EDCF809123058260F7
:10383000E9CF809122058061D5CF809122058062F9
:10384000D1CF809122058064CDCF0E94400F80911E
:1038500022058068C7CF809122058C60C3CF8091FC
:1038600023058360CFCF809122058E7FBBCF8091CF
:103870002305877FC7CF809122058D7FB3CF8091AD
:1038800022058B7FAFCF80912205877FABCF8091C0
:1038900023058E7FB7CF809123058D7FB3CF809195
:1038A00022058F7E9FCF809122058F7D9BCF8091B7
:1038B00022058F7B97CF0E94400F809122058F7742
:1038C00091CF80912205837F8DCF809123058C7FBE
:1038D00099CF80912205992782FF939590FB82F9D9
:1038E00090FB83F97FCF80912305982F909590FBD3
:1038F00080F990FB81F986CF90912205892F8F7BEB
:1039000096FF80646FCF0E94400F90912205892F0F
:1039100097FB87F9805866CF61E08EE090E00E94C7
:10392000703262CF60E0F9CF90912205892F8F7EAF
:1039300094FF806157CF90912205892F8E7F90FF51
:10394000816050CF90912305892F877F93FF8860F6
:1039500059CF89E2E7C389E2F6C38272F801E052E7
:10396000F847EB30F10508F04CC0E652FD4C0C94E2
:103970008B310737FCE71F0709F047C081E00E9441
:10398000280565C080915F0480FF0BC08E7F809307
:103990005F048FE594E0EBD810925E040E94AB08C0
:1039A0007ACB816080935F0461E086958695E3D948
:1039B00072CB811521F020DA6ECB8115E1F312DA9A
:1039C0006ACB811521F08CD966CB8115E1F380D9C2
:1039D00062CB811521F097D95ECB8115E1F388D9AF
:1039E0005ACB811521F0A5D956CB8115E1F396D993
:1039F00052CB811521F0F1D84ECB8115E1F3E3D8FC
:103A00004ACB07372CE71207F9F008373CE71307D2
:103A100021F19801205E32452032310518F59111CF
:103A200021C00F7181E090E0AC0102C0440F551F2E
:103A30000A95E2F78A01642F83E090E00E947032D9
:103A4000802F0E94180527CB81E00E941E0543E0CD
:103A500062E081E00E94A0051ECB82E0911509F48E
:103A60008ECFF3CF4091670480912105282F30E05D
:103A70002095309570E024233723232B19F0482319
:103A8000409367040B375CE7150741F4911509F47F
:103A900002CB0E94FF040E94DE09FDCA003482E5C9
:103AA000180708F056C00032A2E51A0708F058C0FF
:103AB0000115B0E51B0758F50115E0E41E0708F0F5
:103AC00065C0911509F47BC00A35BCE71B0709F4F2
:103AD000EEC008F0D2C00130FCE71F0709F4E5C0D2
:103AE00003302CE7120709F4DAC001153CE713078D
:103AF00009F065C00E94400F8FEF94E3ACE0815065
:103B00009040A040E1F700C000000E94110D980114
:103B1000305521153240A8F6980145E03695279595
:103B20004A95E1F7822F8F702091670430E041E0E1
:103B300050E0082E02C0440F551F0A94E2F72423D8
:103B40003523232B09F4BDCF9111A5CF1092690421
:103B5000EBC29801205C32452032310508F0B1CF2C
:103B6000802F8F712091670430E041E050E0082EF3
:103B700002C0440F551F0A94E2F724233523232B58
:103B800009F49FCF911509F486CA85CFD7011696FF
:103B90008C91803108F095CF911111C0212F2F7099
:103BA00081E090E002C0880F991F2A95E2F72091EA
:103BB000670430E082239323892B09F06CCAD70174
:103BC00017968D919C91009709F475C00E94F0069C
:103BD000D82E192FD7011596BC9015971696AC9034
:103BE000A2948FE0A82280916C048770811509F15E
:103BF000CB2CB114F9F0892F807F803469F080E2FA
:103C00008D0D8830B0F0892F807E803229F4B2E0AB
:103C1000DB1678F0A11469F08091230582FF09C0BA
:103C200082E00E94C90580916C048770CC24C39403
:103C30008111C12C812F82958F70883009F458C171
:103C400008F06DC0843008F04EC0012F0F70823034
:103C500008F476C0107F103211F00295007FD11465
:103C600009F4A2C0F1E0DF1609F404C1B11409F4AB
:103C700010C1A11409F4B4C076C00B354CE7140789
:103C8000C1F080912305002482FF0394802D0C3520
:103C90005CE7150709F093CF0E94970D90CF6FEF67
:103CA0007FEF80E090E00E948A320E945E0F81E008
:103CB000F3CF80E0F1CFF7018581C080D1808115FD
:103CC00069F0C6010E94C112182F682FC6010E9418
:103CD0003605B601812F0E94A61278CFC6010E9438
:103CE0006C05182FF6CF843009F4E5C0C11409F42F
:103CF00030C180916C0480FD2CC1D70115961C92B7
:103D00008695869586950E941E05C7017ED880916E
:103D10006C048695869586950E9428051AC189307F
:103D200009F45BC18A5F8F70823000F7E2EFDE1228
:103D300065C1812F8F71B1105EC10E941E0505C142
:103D4000103110F00295007FB114A9F0011559F05F
:103D500080E28D0D883010F0D11007C0802F0E94B6
:103D6000E4050E94D40D8D2D2DC080916B04802B15
:103D700080936B04F6CF8D2D0E94C00E011509F4BF
:103D8000B5CF80E28D0D883010F0D11004C0802FA7
:103D90000E94EA0506C0009580916B048023809301
:103DA0006B040E94D40DA2CF8091230582FD14C024
:103DB000B11459F0011529F0802F0E94E4050E94EA
:103DC000D40D80E00E94280E91CF80E00E94C00EAA
:103DD000011509F48BCFDBCFB11471F1A11004C030
:103DE000802F0E94180F82CF21E0A21211C01091E3
:103DF0006804802F8123081709F478CF0E94F20A03
:103E00009093700480936F04102B109368046ECF0E
:103E100035E0A3126BCF802F0E94180F802F0E94D5
:103E20004A0B80916A04902F9823091709F45ECFFA
:103E3000802B80936A045ACFA11012C0802F0E9459
:103E40001E0F802F0E944A0B80916A04902F9823A6
:103E5000911509F44BCF0095082300936A0446CFCF
:103E600041E0A41243CF809169048023811509F4B5
:103E70003DCFE4CFB11429F056E0A51608F036CFB7
:103E8000AFCF85E0A81608F031CF802F0E941E0F1B
:103E90002DCFA114D1F399E3D91209C0AFEFB7EE3A
:103EA000E3E0A150B040E040E1F700C000008D2DFC
:103EB0000E94C00E1BCF812F869586958370811539
:103EC00069F0813009F012CF8D2D912F9370B110D0
:103ED00002C080E090E00E94670A08CF8D2D912FEC
:103EE0009370B11002C080E090E00E943F0AFECEC5
:103EF000812F837081113AC0B11027C04D2D42959A
:103F000046954770440F440F8D2D8F70042E01C0CD
:103F1000880F0A94EAF72D2D2071D4FE07C02FE0F8
:103F200030E001C0220F4A95EAF7209516951695C4
:103F300013701230B1F0133091F030912005113030
:103F400069F0822B83230E9418050E94300A0E9488
:103F5000120560E0C7010E94EB12ADC8832B822BD3
:103F6000F2CF822B909120058927EDCFB11451F12A
:103F700010FFEBCF4D2D429546954770440F440FEF
:103F80008D2D8F70042E01C0880F0A94EAF72D2D15
:103F90002071D4FE07C02FE030E001C0220F4A9507
:103FA000EAF72095169516951370123089F01330A4
:103FB00069F030912105113041F0822B83230E945A
:103FC0001B05C3CF8230B0F6C0CF832B822BF7CF37
:103FD000822B909121058927F2CF1F70B11439F0FF
:103FE000812F0E941E058D2D0E94180FAECF8D2DA2
:103FF0000E941E0F812F0E942805A7CFF3EFDF1626
:1040000080F420EFD216E1F031EFD316A1F0B11415
:1040100009F460C0A11409F45AC08D2D0E94280E25
:1040200094CF43EFD416F1F054EFD512F0CF809136
:10403000230582FD23C0812F8F71B114E1F27DCE63
:10404000B11469F085E0A81608F07FCF1F7181E0F8
:1040500090E0012E01C0880F0A94EAF7BACF96E0EB
:10406000A916F2CF80E0B11409F4A9CF1F7181E045
:10407000012E01C0880F0A94EAF7A1CFB114C1F054
:1040800080916C048770843049F410926C04109213
:104090006E0410926D04812F8F71ADCFA5E063E0A7
:1040A000AA1608F052CF812F8F710E94360B4DCF88
:1040B000B5E0AB1640F010926C0410926E041092B2
:1040C0006D0464E0F0CF81E00E94C9053ECF812FEE
:1040D0008F7133CEA114F9F2E9E3DE1209C0FFEFCC
:1040E00027EE33E0F15020403040E1F700C00000FF
:1040F0008D2D0E94C00E29CF0337FCE71F073FCA52
:10410000809169040631BCE71B0709F026CC8A7A46
:1041100091E0811101C090E090935C04811509F455
:1041200018CC85E30E948F0A0E94D40D0C944B1882
:104130000631ECE71E0709F01CCC80915C04811568
:1041400009F409CC85E30E94C30AEECFA0E0B0E0F9
:10415000ECEAF0E20C94B33180914B03803108F02B
:1041600049C080914A03811509F444C0C091FC0202
:1041700089E0D82E8091FB028C17E1F1EC2EF12C16
:10418000DC9EE0011124FE01E350FD4F8481811586
:10419000B1F1918180914603981331C09081809153
:1041A000450398132CC08581811129C00281138198
:1041B0008091470390914803081B190B60E085E448
:1041C00093E00E94EB120E943C1508171907B8F4FF
:1041D00080914B038F70806180934B03CD5FDC4FE8
:1041E00088818F708061888385E493E00E94051741
:1041F0000E94BF05CDB7DEB7E7E00C94CF31E701F1
:104200002196C770B7CFAFE0B0E0E9E0F1E20C94DF
:10421000AB318C0186E0F801DE011A9601900D9217
:104220008A95E1F7F801F580E48085E4882E83E043
:10423000982E80914903811117C0E11491F0F11477
:1042400009F480C1C8010E941A13811509F47AC1CA
:1042500089E0F801A5E4B3E001900D928A95E1F7B9
:1042600075DFFF24F3946AC0A280B380D0904A0324
:1042700080914703909148033501681A790AD11457
:1042800009F411C1C080518060E085E493E00E9490
:10429000EB120E943C156816790608F0B6C0E114CE
:1042A00001F380914603F8019181E0904B03F0E126
:1042B000EF1608F064C0981320C090914503F801F0
:1042C000808198131AC020914C0330914D0387814F
:1042D00090852817390789F4F1104BC08E2D8F7007
:1042E000806180934B0385E493E00E9405178091E1
:1042F0004B03F8018683F12C21C0F1103AC040E055
:10430000652D8C2D0E94CC0C40E0652D8C2D0E94DB
:10431000CC0CF82E8111EFCF8A859B850E940D135E
:10432000292F22952F70903470F49F702230A0F0C6
:104330009115B1F0F8019681903190F48F2D2F9660
:10434000EFE00C94C7312A5F2F70223068F0C8016B
:104350000E940517FD2CF2CF911511F0811571F314
:10436000805E883058F3F3CF803F40F3815F833025
:10437000F9CF80914B03816080934B03BCCF98139E
:104380001EC090914503F8018081981318C02091B8
:104390004C0330914D03878190852817390779F4B4
:1043A000F1100DC0E682C8010E94051789E0F801EE
:1043B000A5E4B3E001900D928A95E1F752CFC801D0
:1043C0000E941A13811509F4BDC0F11409F4BAC092
:1043D00080914B03803208F43BCF8091450390914C
:1043E00046039A838983BC82AB82809149038D8383
:1043F0001E82EF8280914C0390914D0399878887AC
:10440000CE0101960E94051723CFD0904B03F0E117
:10441000DF1650F485E493E00E94051789E0F4016B
:1044200011928A95E9F767CFE11409F41ACF9091B8
:104430004603F801818198131AC090914503808149
:10444000981315C020914C0330914D0387819085BE
:104450002817390761F4F1100AC0D682C8010E94FA
:10446000051789E0F40111928A95E9F7FACEC8019F
:104470000E941A13811509F465C0F11409F462C091
:1044800080914B03803208F4E3CE809145039091F4
:1044900046039A838983BC82AB82809149038D83D2
:1044A0001E82DF82A7CF60E085E493E00E94EB12DA
:1044B0000E943C156816790608F0B0CFE11409F4A3
:1044C000D0CEF11409F43EC090914603F8018181E9
:1044D00098132EC0909145038081981329C0209194
:1044E0004C0330914D03878190852817390701F5DA
:1044F0008091470390914803A81AB90AF8ECAF16C7
:10450000B10408F053CF80914B0380FD4FCF803131
:1045100008F44CCFF8018683982F907F903F09F4E0
:1045200042CF982F907F905F8F70892B86833BCFEF
:10453000C8010E941A1381118BCE80914B038160B8
:1045400080934B03C8010E9405178BCEA2E1B0E017
:10455000ECEAF2E20C94B6310A871B872C873D8780
:104560004E875F87688B798B8A8BCE010A964BDEEC
:10457000811128C02091FB023091FC0289E0FE01EC
:104580003A96DE01119601900D928A95E1F78E859B
:104590008115C1F0822F90E0019687709927381716
:1045A0001906D9F099E0929FD0011124A350BD4F74
:1045B000FE01319601900D929A95E1F78093FB02EE
:1045C0000E94BF0519E08091FC029091FB028913C3
:1045D00012C06296E4E00C94D2310E94400F109217
:1045E000FB021092FC0289E0E5E4F3E0DF011D929A
:1045F0008A95E9F7E7CF189FC001112483509D4F9A
:1046000002DE811531F38091FC0290E00196877003
:1046100099278093FC02D7CFEF92FF920F931F93BD
:10462000CF93DF9380911D05E0911602CDE08111BB
:1046300030C0CDB7DEB7E6E00C94D031D1E0DE0F6C
:10464000D0931602EE2EF12CCE9FF0011124EB54E4
:10465000FB4F84818115E1F087819085892B21F4BE
:1046600081859285019651F40081118122813381E7
:104670004481558166817781808568DFCE9DF00118
:10468000CF9DF00D1124EB54FB4F148210926B045C
:10469000ED2F80911D05E81788F210921D051092EC
:1046A0001602C7CFA4E0B0E0E8E5F3E20C94A9312C
:1046B0002091B404298397E0992E01E010E02DE0C9
:1046C000322E34E0532E882483948091B304998150
:1046D000891307C0A1DF0E94A1092496E1E10C948F
:1046E000C5319981892F90E09C838B83FC01EE0F6B
:1046F000FF1FE755FB4F80819181989ED001999EC5
:10470000B00D1124FD01EF58FB4FFA83E98324819A
:1047100021115BC060901D05E5EBF4E060E070E006
:10472000712C661508F04FC0A384B484A981BA81A6
:10473000CD90DC902FEF3FEF412C442D50E07601DF
:10474000E40CF11CE40CF11CD701ED90FC90E11499
:10475000F10439F0AE14BF0409F0A90143949A01A1
:10476000ECCF2F3F3207D1F1D80102C0AA0FBB1FF7
:104770002A95E2F77A2A9801042C02C0220F331FEF
:104780000A94E2F7A901415051097416150629F55A
:10479000369EF001379EF00D1124EB54FB4F989E8E
:1047A000D001999EB00D1124AF58BB4F12962D9198
:1047B0003C9113973087278354821082118292870D
:1047C000818715968C920E94B2098B819C810196FB
:1047D0009A8389838370898378CF14826F5F7F4F38
:1047E0003D969FCF10921F0510921E0510921B013F
:1047F0008091B3048093B4040E94A1090DCFACE171
:10480000B0E0E5E0F4E20C94A8314B8B5C8B6D8B4F
:104810007E8B8F8BB92E988FA92E911110926B04DD
:10482000188A198A1A8A86E0FE017396DE011A96A2
:1048300001900D928A95E1F75F888091230582FFB0
:104840001FC00E94F20A20916D0430916E04821BF9
:10485000930B8838934138F080916C0482FD03C03B
:1048600082E00E94C9050E94F20A20916F043091F3
:104870007004821B930B8838934110F00E94F2055C
:104880005114D9F05E86BF8661E0CE010A960E947F
:10489000EB1261E0CE010A960E94EB1261E0CE01BC
:1048A0000A960E94EB124C0180356CE7960791F452
:1048B000A11419F181E080931B015E86BF860A85F1
:1048C0001B852C853D85452D5B2D688979898A89D5
:1048D0003DDECDC081359C4721F4A11471F082DF0B
:1048E000ECCF82E588168CE7980639F4A11429F0FC
:1048F00080911B018111F3CFDDCF41E7E42E44E02D
:10490000F42E412C612C712CD7016D917C91CC241B
:10491000CA94DD24DA9480E0282F30E0FB01E80F10
:10492000F11DE80FF11D408151814115510539F00C
:104930008416950609F096018F5F6901EDCF10E0AE
:10494000BFEFCB16DB0609F44EC0F701448110918E
:104950001B01411110E0D70115963C901597169652
:104960009C911697A11409F405C1111509F402C10F
:10497000311017C021E030E00C2C01C0220F0A9446
:10498000EAF7922B16969C932091B1043091B204D1
:104990002233310530F422E330E03093B204209327
:1049A000B104E1E0F0E002C0EE0FFF1F8A95E2F7EC
:1049B000CF010197D70116962C912817190699F463
:1049C000C0901E05D0901F05C114D10409F453C036
:1049D0000E94F20A8C199D09C39708F44CC081E02B
:1049E000F701848311E0412ABFEF6B1A7B0AE7E0ED
:1049F000EE0EF11CF8E06F16710409F085CFA114DA
:104A000009F417C1411409F414C10E94F20A9093E9
:104A10001F0580931E0580911D05883040F591E0AB
:104A2000980F90931D0599E0FE013A96DE011196CC
:104A300001900D929A95E1F75D82BE822DE0829FF2
:104A4000C00111248B549B4F29E0FE013196DC01FB
:104A500001900D922A95E1F72FEF3FEFDC011A96B6
:104A60003C932E9319971C969C928E921B976C9652
:104A7000E2E10C94C4312091B4048091B304922FEC
:104A8000E0E0F0E001E0281709F448C0422F50E0D0
:104A9000FA01EE0FFF1FE755FB4F2080318037E012
:104AA000329DF001339DF00D1124EF58FB4F6081D2
:104AB00071817C8F6B8FB0E030E0A0E0EB8DFC8DDE
:104AC000EA0FF11DEA0FF11DC080D180C114D1049D
:104AD000E1F0F7010190F081E02DFA8FE98F30E0ED
:104AE00007C0E1E0C616D70609F0E0E0BE2B3F5F45
:104AF000E98DFA8DE30FF11DE30FF11D60817181E6
:104B00006115710571F7AF5FD9CFB11581F13A1712
:104B1000C8F4E1E0D7011496EC93F7019093B40444
:104B2000EE15FF0509F45FCF90E0FC01EE0FFF1FCB
:104B3000E755FB4F718260820196837099278093BD
:104B4000B30451CF37E0329DF001339DF00D1124B5
:104B5000EF58FB4F0483EE15FF05F9F2291302C04D
:104B60009F5F93709A012F5F3F4F23708CCFE0E0DF
:104B7000F0E0F8CF292F30E0311024C061E070E080
:104B800002C0660F771F8A95E2F7CB0101972817BD
:104B9000390791F010E0E1E0F0E002C0EE0FFF1FF6
:104BA000CA94E2F76F01C094D70116968C911697BC
:104BB0008C2116968C9317CF411569F3C3010E947F
:104BC000B209E8CFA9010C2C02C0559547950A946B
:104BD000E2F7C901019782239323892B39F540FF1E
:104BE00025C0D70112968D919C91892BD1F087E039
:104BF000FE013196DF011D928A95E9F70E94F20AC3
:104C00009C018B839C8384E08D83F7019281838157
:104C1000792F9887898709811A8144E05E816F81A5
:104C200095DCD70115961C92132DB5CF142F11705A
:104C3000B2CF9091B4048091B304981731F032DD73
:104C4000B1E04B1609F413CF38CEE6DC10921F0505
:104C500010921E050E94A109F3CFA6E0B0E0E3E3A5
:104C6000F6E20C94B6310E94F20A8C018091CF02D8
:104C70009091D0028017910771F019821A820E94D8
:104C8000F20ABC0149815A8180E090E0B8DD1093BE
:104C9000D0020093CF022696E4E00C94D231A6E035
:104CA000B0E0E5E5F6E20C94B6318C019093CC02CD
:104CB0008093CB02011580E21807B0F4C801805E32
:104CC0009109089728F064E27FE00115110511F4BD
:104CD00068E17FE0C8010E94D004802F0E94280E66
:104CE0002696E4E00C94D23180EF89838A830E9477
:104CF000F20A8160BC0149815A8181E091E07FDD47
:104D0000EFCFA6E0B0E0E7E8F6E20C94B6318C0114
:104D10009093CC028093CB02011580E21807B0F487
:104D2000802F0E94C00EC801805E9109089728F06C
:104D30006DE27FE00115110511F46EE17FE0C8011D
:104D40000E94D0042696E4E00C94D23180EF89834F
:104D50008A830E94F20A8160BC0149815A8181E004
:104D600090E04DDDEFCFCF93DF93D82FC92F97DFA2
:104D70008D2F9C2FC6DFDF91CF9108950F931F9346
:104D8000CF93DF938C01862F69EC73E00E94271587
:104D9000892B91F4C091C903D091CA03209761F087
:104DA000F8018281833039F4CE01DDDFCE01DBDF13
:104DB000CE01D9DF01C0E0F7DF91CF911F910F91B4
:104DC00008950F931F93CF93DF938C01EB0169EC50
:104DD00073E08C2F0E942715892B09F057C0FE0124
:104DE000FF27D80112968C911297EF56FD4F813014
:104DF000A9F415968C9182FD4EC080FF4CC082E0D4
:104E000080838091CB039091CC030097B9F480917B
:104E1000C9039091CA030097C9F110C08230A1F56F
:104E200015968C9182FD26C080FD0AC083E08083A8
:104E30008091CD039091CE030097F1F030DF26C032
:104E400084E080838091CF039091D0030097B1F7E5
:104E50008091C9039091CA03009701F184DF80918A
:104E6000CB039091CC03009749F78091C9039091AF
:104E7000CA03E4CF85E080838091C9039091CA037F
:104E8000009721F070DFF1CF86E08083DF91CF9132
:104E90001F910F91089581E08083B9CF8091CB035A
:104EA0009091CC03B8CF0F931F93CF93DF938C01D6
:104EB000EB0169EC73E08C2F0E942715892B71F4AC
:104EC000DD27CF56DD4F8881F801128218828330AA
:104ED000E9F048F4813059F0823081F0DF91CF91D0
:104EE0001F910F9108958430B1F08530B9F780910A
:104EF000C9039091CA03009789F306C08091CB0340
:104F00009091CC03009799F3FCDEE8CF8091CD031C
:104F10009091CE03F7CF8091CF039091D00300976B
:104F200099F72091C9033091CA038091CB039091E6
:104F3000CC0321153105F9F2009731F7C901E4CF0F
:104F4000A0E1B0E0E6EAF7E20C94AA31FE01319666
:104F500080E1DF011D928A95E9F70EE010E099E209
:104F6000A92E93E0B92E27ED422E512C612C712CE5
:104F70004F0173016201B1E14B16510461047104E8
:104F80001CF080E1C82ED12CA601B501C4010E94FD
:104F90006132AC0CBD1C0D2C000CEE08FF084C1847
:104FA0005D086E087F080150104019F76096E0E137
:104FB0000C94C6316FEF85E290E00E9470326FEF83
:104FC00086E290E00E9470326FEF87E290E00E94EC
:104FD000703260E088E290E00E9470320E941D14FE
:104FE000AFDF64EE85E290E00E9470326EE286E20E
:104FF00090E00E94703268E987E290E00C94703291
:105000008F929F92AF92BF92CF92DF92EF92FF92D8
:105010000F93CF93DF9388E090E00E9457324B01CB
:105020005C01CFE5D4E068839982AA82BB821C82AE
:105030001D821E821F8283E290E00E944F32282F41
:1050400030E040E050E060E070E080E090E000E2BE
:105050000E94DF31282939294A295B29288339838D
:105060004A835B836C837D838E839F83DF91CF91A3
:105070000F91FF90EF90DF90CF90BF90AF909F90F7
:105080008F900895AAE0B0E0E8E4F8E20C94AC3127
:10509000FE0131968AE0DF011D928A95E9F79DE4D1
:1050A000A92E91E0B92E8F013F01EE24E394F12C5B
:1050B00030E6C32E31E0D32EF50181915F018F3FA1
:1050C00009F444C0F894E82FE295EF70F0E021A1D4
:1050D0008F70A70102C0440F551F8A95E2F7CA01DD
:1050E000922F982B91A392A18095892382A37894E3
:1050F00000C0E2E5F1E021E030E0812C912C41910B
:105100004F3F79F0A42FA295AF70A05EB0E08C91D4
:1051100090E04F7002C0959587954A95E2F780FF21
:105120003BC080E090E0882A992A220F331FCE16D8
:10513000DF0629F7F50182918F3F11F00E94EE07FB
:1051400050EA5A95F1F7D8018D929C920E5F1F4F4D
:10515000B2E5AB16B1E0BB0609F0AECF4AE050E0D5
:10516000B30189E992E00E942B32892BB9F08AE0E1
:10517000F301A9E9B2E001900D928A95E1F781E08F
:105180008093F8010E94F20A9093F7018093F60150
:105190002A96EEE00C94C831C901C5CF8091F80180
:1051A0008115B1F30091F6011091F7010E94F20A06
:1051B000801B910B059760F34AE050E069E972E0CB
:1051C0008EEB92E00E942B32892B49F08AE0E9E9CC
:1051D000F2E0AEEBB2E001900D928A95E1F7109209
:1051E000F801D6CFCDB7DEB7AC970FB6F894DEBFD7
:1051F0000FBECDBF85B7806885BF85B7806885BF86
:1052000084B7877F84BF0FB6F894A895809160001B
:10521000886180936000109260000FBE80E890E08B
:105220000FB6F89480936100909361000FBE81E007
:1052300080931A018CEE97E09093CD018093CC017E
:105240000E9441090E94A3140E94E7140E94150CB9
:105250000E94720C8091E20084608093E200789456
:105260008091CA02811599F08091E9001091EC00BB
:105270008F70179511271795182B1092E9008091C0
:10528000E80083FD0E94730F1F701093E90082E015
:1052900084BD93E095BD9AEF97BD80936E000E9408
:1052A0005C13811101C086DE0DE411E0D8018D91FF
:1052B0008D018F3F11F00E94EE07B1E002351B0710
:1052C000A9F702E511E020E6E22E21E0F22EF80136
:1052D00081918F018F3F11F00E94EE07E016F106D9
:1052E000B1F78AE0EEEBF2E0DF01282F1D922A955C
:1052F000E9F7E9E9F2E0DF011D928A95E9F780E03C
:1053000090E00E945C32833E9E4F21F40E945C1329
:1053100081112AC063EE7EEF80E090E00E948A3225
:1053200060E082E090E00E94703281E0809320058E
:1053300061E083E090E00E94703260E074E184E01C
:1053400090E00E948A320E94D81534DE40E050E09E
:10535000BA018FE090E00E94823240E050E0BA0152
:1053600083E190E00E94823282E090E00E944F321E
:105370008093A80284E090E00E945C329093230521
:10538000809322057FDEEFEFF6E721E0E150F04069
:105390002040E1F700C0000075DE8091BE0280FF72
:1053A00008C06FEF7FEF80E090E00E948A320E9499
:1053B000110D83E090E00E944F320E941805549A2C
:1053C0005C9A8091A30281111EC08FE594E018DEE3
:1053D00080915F04843028F40E94D8158FE594E012
:1053E0000FDE0E949D0810925E040E949409809135
:1053F0005F0480FF05C060E0869586950E94BB161D
:1054000081E08093A3028BE091E09093F20280937D
:10541000F1028091CA028530E9F48091CA02853098
:1054200009F46FC00E94400F0E94300A0E941205CA
:105430001092A6028091A502811551F080915F041F
:10544000816080935F0460E0869586950E94BB161C
:105450000E94A41617DE99EAA92E92E0B92E0EEB4F
:1054600012E0D801F501219131918D919D9143EB8D
:1054700052E04E175F0709F491C02817390799F3D6
:105480008EEB882E82E0982E512CD401ED90FD9069
:105490004D01F501619071905F016E147F0451F12F
:1054A0006E247F24412CCC24C394D12CC6018621A8
:1054B0009721892BB1F049825A820E94F20A9C837B
:1054C0008B83F1E0FD8391E096012E213F21232B78
:1054D00009F490E09E8349815A816B817C818D81A2
:1054E0008ED94394CC0CDD1C2EE04212DFCFF501A7
:1054F000F292E292539435E05312C7CF0E945F0BB1
:1055000052C08091CA02843009F43BC080E00E94FE
:10551000120510925E048091A60281110EC031E046
:105520003093A60280915F04982F91709093A5020A
:105530008E7F80935F040E94AB081092A40248E122
:1055400050E080E40FB6F894A895409360000FBE39
:105550008093600083B7817F846083BF83B781605D
:1055600083BF7894889583B78E7F83BF0FB6F894F6
:10557000A89580916000886180936000109260001F
:105580000FBE80DDEEEBF2E081919191892B09F065
:1055900013C592E0E83CF907B9F73FCF2817390760
:1055A00009F06ECF5ADBC0905704D0905804C11454
:1055B000D10439F1A0905904B0905A040E94F20A23
:1055C0007C01EA18FB08C6010E943C158E159F0558
:1055D000C0F42091570430915804C9019927287FBD
:1055E0003327232B09F0CBC0F4E0880F991FFA95DD
:1055F000E1F789529C4FDC0115962C9122FF0E9405
:10560000521280911B01811511F1E0901E05F0905E
:105610001F05E114F104D9F00E94F20A8E199F09C6
:105620002091B1043091B2042817390780F4909189
:10563000B4048091B304981709F4A4C033D810922D
:10564000B2041092B10410921F0510921E058091B1
:10565000D303811569F00E94F20A2091D40330919E
:10566000D503821B930B8F3F9F4710F40E94370F87
:1056700080915E048115D9F180915D04E0915F0411
:10568000E695E695E81BE093B502823009F083C009
:10569000F0E0E756F94FE491EE2EF12CEBEFCE2E31
:1056A000E8E0DE2E8091B602811561F01092B6021C
:1056B0000E94F20A9093B4028093B3021092B8024F
:1056C0001092B7020E94F20A2091B3023091B40204
:1056D000821B930B8F3F9F4750F42E0D3F1D30933D
:1056E000B4022093B30283EB92E0F60109950E9485
:1056F000300AF82E8091B902F81639F0F092B9020A
:105700000E945F0B8F2D0E9412058091CA02843087
:1057100009F07FCE83E08093E9008091E80082FF6A
:1057200078CE8091E80090E085FF06C00E94E40BEF
:10573000811509F454C091E08091E8008B77809343
:10574000E800911509F465CEE090CD02F090CE020C
:10575000E981E114F10409F461C0EE3F09F081C070
:105760008A81833020F08550833008F07AC0EA8146
:10577000EE3008F076C0F0E0EB51FD4CCCC580E097
:1057800090E039CF0E940C2310921F0510921E0545
:105790000E94A1095CCF863059F4F0E0EA56F94F37
:1057A000E491EE2EF12C7CEEC72E78E0D72E7ACF46
:1057B00040EDE42E47E0F42E57E0C52E58E0D52EFC
:1057C000893009F06FCFE695F0E0ED56F94FE4919E
:1057D000EE2EF12C6EE0C62E69E0D62E63CF30E2BD
:1057E000C32ED12C9E012F5F3F4F79018091E8009D
:1057F00085FD0AC08091E8008B778093E8000E94C5
:10580000E40B811599F397CF8091F100D7018D9327
:105810007D01B1E0CB1AD10849F78DCFE43148F4CE
:10582000E11551F0E150E33138F4F0E0ED50FD4C7A
:1058300072C5EE3F09F49BCF8FEF898312C01A82A5
:1058400089E08B830EC08A81823081F08330B1F091
:10585000813091F70E945F0B74D56B837C838D83BD
:105860009E83CE0101960E94340CD3CD88E290E055
:1058700016D61B821C821D828E83F3CF8091C802B4
:105880009091C902892B69F3FE013196D8018C9160
:1058900011969C910E5F1F4F928383833296B2E0E4
:1058A000083C1B0799F7DDCF8A81823029F66B818E
:1058B0007C818D819E8145D588E290E011D6D1CF43
:1058C0004C816B818A810E947712982789279827BB
:1058D0009E838D83C6CF2D813E8132272327322799
:1058E0004C816B818A810E94AD0DBBCF0E941D143B
:1058F000B8CF8A81823891F1B0F48038E9F08138EC
:1059000009F0AFCF60E08B810E94BB169B81809134
:105910005F0491111AC08E7F80935F0410925E0421
:105920000E94AB089ECF833809F09BCF20E04091C6
:1059300062046C818B8106C020E04B816091610420
:10594000809160040E94F7158CCF816080935F0482
:1059500060E0869586950E94BB1683CF8B818093ED
:1059600063047FCF8A818238E1F060F48038A1F04F
:10597000813809F076CF80915F0480FF10C0869552
:1059800086955FCF833809F06CCF809160048B835C
:10599000809161048C8365CF8091620452CF80E056
:1059A00050CF809163044DCF0E949D088FE594E015
:1059B0000E94B71556CF80E18A8353CF1A8287EDB4
:1059C00040CF8C818D3108F04CCF8A809B80982409
:1059D00089249824A12CB12C8E010F5F1F4F7801D0
:1059E000E80EF11CE016F10609F43BCF80E0E7ED8C
:1059F0008E169104A104B10420F4C401875D9C4F6C
:105A00004ED5D80114968C930F5F1F4FBFEF8B1AA2
:105A10009B0AAB0ABB0AE6CF8091C8029091C902EB
:105A2000892B09F41ECF8C818D3108F01ACF882E76
:105A3000912CA12CB12CCA80DB80DC24CD24DC2469
:105A4000E12CF12C8E010F5F1F4F412C512C3201A4
:105A5000481459046A047B0408F003CFE7EDCE161E
:105A6000D104E104F10438F4D80114966C91C60114
:105A7000875D9C4F35D5BFEF4B1A5B0A6B0A7B0ADB
:105A8000EFEFCE1ADE0AEE0AFE0A0F5F1F4FE0CFDD
:105A900057DAE7CE84E090CF8C818D3108F0E1CEEB
:105AA000882E912CA12CB12CCA80DB80DC24CD2443
:105AB000DC24E12CF12C412C512C32018E010B5FA6
:105AC0001F4F481459046A047B0408F0CACE80E0D2
:105AD000F0E3CF16F2E0DF06E104F10418F4C601AA
:105AE0008996DDD4D8018D938D01BFEF4B1A5B0AE7
:105AF0006B0A7B0AEFEFCE1ADE0AEE0AFE0AE1CF4E
:105B00002C81022F10E02D3108F0ABCE8A819B81D1
:105B10009827892798272C01612C712C8033F2E07B
:105B20009F0708F09ECE822E912CA12CB12C40E331
:105B300052E060E070E044195509660977094217A0
:105B400051056105710508F48CCE2091C802309191
:105B5000C902232B09F03EC01C0129E2220E311C90
:105B600080FBEE24FF24E0F880FF0BC0889697D4DA
:105B70009D8189279827892781159C4711F48FEFEC
:105B80008D83D501C401840D951DA61DB71D80FF11
:105B900019C0680141E0C41AD108CE0105968C0DE8
:105BA0009D1D9CA78BA7C101800F911F78D4ABA529
:105BB000BCA59C9181159C4721F48FEFEBA5FCA51A
:105BC00080838601FE013196EE0DFF1D2FEFE0165A
:105BD000F10638F08E010F5F1F4FC12CD12C7601DA
:105BE00025C09481858181159C4711F424832583E8
:105BF00042E0E40EF11C3296EACF50E3451652E043
:105C000055066104710430F4D80114966C91C201F8
:105C1000899666D4BFEFCB1ADB0AEB0AFB0AEFEFDB
:105C20004E1A5E0A6E0A7E0A0F5F1F4FC814D9040F
:105C3000EA04FB0410F315CE8091C8029091C902CA
:105C4000892B09F40ECECE0101960E94340CFFEF91
:105C500021EE34E0F15020403040E1F700C0000078
:105C6000A6CB88E0ECE1F1E0DE01919601900D9287
:105C70008A95E1F7FE0132968FE1DF011D928A9548
:105C8000E9F786E0898388E07F96DE01159601902A
:105C90000D928A95E1F7E5CD88E6898382E08A83D3
:105CA0001B821C82DECD8B819C81092E000CAA0BED
:105CB000BB0B25E0880F991FAA1FBB1F2A95D1F7A0
:105CC000AC01BD01405E5F4F6F4F7F4F48175907D2
:105CD0006A077B0708F4C5CD8836E2E09E07A10578
:105CE000B10508F0BECD4936F2E05F0761057105E8
:105CF00020F048E652E060E070E0481B590BBC0120
:105D00006356794FCE01019690D3ABCD4AE150E076
:105D10006FEF70E0CE010796ABD38091C802898304
:105D2000EA821B821C8282E08D838DE0A5CD81E01A
:105D300090E09093CE028093CD0282E390E0909326
:105D4000BD028093BC020E94F20A9093BB02809332
:105D5000BA0287CDE114F10481F1D090BE02C09067
:105D6000C3020091BA021091BB020E94F20A801B8A
:105D7000910B8536910540F1C5FE26C0D0FE24C0AA
:105D80000E94F20A9093BB028093BA028091BC02F7
:105D90009091BD0201979093BD028093BC02892B24
:105DA00061F41092CE021092CD0281E090E09093C7
:105DB000C9028093C802E12CF12C8091C80289832A
:105DC000EA828091BC023DCD82E390E09093BD02D7
:105DD0008093BC02F2CF1092C9021092C80241CD4A
:105DE00040E250E06FEF70E0CE01019641D339CD33
:105DF000EB81E93008F035CDF0E0EA5FFC4C8BC276
:105E0000FE0133968DE1DF011D928A95E9F788E066
:105E100089838A838C8383E088A323CD8C819AE055
:105E2000F92E8E010F5D1F4FF8012F2D11922A952B
:105E3000E9F7B8010E9427158983F801DE0112965F
:105E400001900D92FA94E1F70CCD1C818AE0FE01DD
:105E50003596DE01919601900D928A95E1F789A120
:105E60009AA10E9434099AA389A38BA19CA10E94A4
:105E700034099CA38BA38DA19EA10E9434099EA3EB
:105E80008DA38FA198A50E94340998A78FA38FEFA7
:105E9000183060F43AE0139FB0011124675A7D4F27
:105EA0004AE050E0CE01819639D380E089830E9498
:105EB0004109D7CC2C816AE0CE018196DC01E62F26
:105EC0001D92EA95E9F7283080F4629FB001112411
:105ED00067557D4F4AE050E0D2D280E089838AE066
:105EE000FE01B196DE011296D2CE8FEFF7CF1C8164
:105EF0008AE0FE013596DE01919601900D928A9519
:105F0000E1F789A59AA50E9434099AA789A78FEF7E
:105F1000183060F4FAE01F9FB001112467557D4FDF
:105F20004AE050E0CE018196F9D280E089830E9458
:105F3000A31497CC2C8166E0CE018196DC01E62F7C
:105F40001D92EA95E9F7283060F4629FB0011124B0
:105F500067507D4F46E050E092D280E0898386E032
:105F6000BFCF8FEFFBCF1C8186E0FE013596DE01AF
:105F7000919601900D928A95E1F789A19AA10E94CC
:105F800034099AA389A38BA19CA10E9434099CA3E4
:105F90008BA38FEF183060F4F6E01F9FB00111243F
:105FA00067507D4F46E050E0CE018196B7D280E049
:105FB00089830E94E71455CC8091A702811509F4CA
:105FC0002CCAA0E1A9BDB2E1B9BD09B400FEFDCF64
:105FD0008091D8008F7D8093D8008091E00082600E
:105FE0008093E0008091E00081FDFCCF0E94400F93
:105FF00014CA1F921FB61F9211248F939F93AF93C1
:10600000BF938091A402811113C080910E029091E0
:106010000F02A0911002B09111024196A11DB11D75
:1060200080930E0290930F02A0931002B09311027E
:10603000BF91AF919F918F911F901FBE1F90189598
:1060400078941F921FB61F9211248F939F93AF9342
:10605000BF9380910E0290910F02A0911002B09117
:1060600011020196A11DB11D80930E0290930F02A3
:10607000A0931002B0931102BF91AF919F918F91A5
:106080001F901FBE1F9018951F920F920FB60F9270
:1060900011242F933F934F935F936F937F938F932D
:1060A0009F93AF93BF93EF93FF938091E10082FFA3
:1060B00009C08091E20082FF05C08091E1008B7FE2
:1060C0008093E1008091DA0080FF24C08091D800A5
:1060D00080FF20C08091DA008E7F8093DA0080916B
:1060E000D90080FFA9C080E189BD82E189BD09B4E2
:1060F00000FEFDCF81E08093CA028091FD018111F5
:1061000009C00E94150C0E94720C8091E20084600C
:106110008093E2008091E10080FF1AC08091E2004C
:1061200080FF16C08091E2008E7F8093E200809114
:10613000E20080618093E2008091D80080628093C9
:10614000D80019BC85E08093CA0283E080931A01CD
:106150008091E10084FF2FC08091E20084FF2BC07A
:1061600080E189BD82E189BD09B400FEFDCF809147
:10617000D8008F7D8093D8008091E1008F7E80933E
:10618000E1008091E2008F7E8093E2008091E20046
:1061900081608093E2008091FC01811509F452C076
:1061A00084E08093CA028091CA02843009F052C010
:1061B00082E080931A018091E10083FF2CC08091DE
:1061C000E20083FF28C08091E100877F8093E10097
:1061D00082E08093CA021092FC018091E1008E7FE0
:1061E0008093E1008091E2008E7F8093E2008091B5
:1061F000E20080618093E20042E060E080E00E9483
:10620000420C8091F00088608093F00081E08093E0
:106210001A0180931901FF91EF91BF91AF919F9166
:106220008F917F916F915F914F913F912F910F903F
:106230000FBE0F901F90189519BC1092CA021092B1
:10624000FD0168CF8091E30087FF02C083E0A9CF02
:1062500081E0A7CF81E0ADCF1F920F920FB60F92D2
:106260001124EF92FF920F931F932F933F934F931D
:106270005F936F937F938F939F93AF93BF93CF93CE
:10628000EF93FF9309EE10E0F8018081C091EC00DC
:106290008F70C795CC27C795C82B108280EFE82E4A
:1062A000F12CF7018081877F808378940E94730F9F
:1062B000F8011082F701808188608083CF70F80137
:1062C000C083FF91EF91CF91BF91AF919F918F913B
:1062D0007F916F915F914F913F912F911F910F91FE
:1062E000FF90EF900F900FBE0F901F901895AA1B74
:1062F000BB1B51E107C0AA1FBB1FA617B70710F0B1
:10630000A61BB70B881F991F5A95A9F780959095E2
:10631000BC01CD010895EE0FFF1F0590F491E02D13
:106320000994082E817006940694811D0694811D9F
:106330000694811D0694811D0694811D0694801D7E
:10634000089569279627692778278727782708954A
:106350002F923F924F925F926F927F928F929F9275
:10636000AF92BF92CF92DF92EF92FF920F931F9363
:10637000CF93DF93CDB7DEB7CA1BDB0B0FB6F89414
:10638000DEBF0FBECDBF09942A88398848885F8454
:106390006E847D848C849B84AA84B984C884DF80C5
:1063A000EE80FD800C811B81AA81B981CE0FD11DA9
:1063B0000FB6F894DEBF0FBECDBFED010895002EDD
:1063C000083090F0982F872F762F652F542F432F6A
:1063D000322F22270850F4CF220F331F441F551F9E
:1063E000661F771F881F991F0A95B2F7002D089521
:1063F00097FD1094002E083098F00850232F342F6A
:10640000452F562F672F782F892F912DF4CF159474
:1064100097958795779567955795479537952795DC
:106420000A95AAF71124002D0895FB01DC0102C092
:1064300005900D9241505040D8F70895FC0141500D
:10644000504030F001900616D1F73197CF010895F2
:10645000882799270895FB01DC0104C08D910190E4
:10646000801921F441505040C8F7881B990B0895BA
:10647000DC0101C06D9341505040E0F70895DC010C
:10648000CB01FC01F999FECF06C0F2BDE1BDF89A3F
:10649000319600B40D9241505040B8F70895F999E3
:1064A000FECF92BD81BDF89A992780B50895A6E1E7
:1064B000B0E044E050E0E5CFA8E1B0E042E050E0D9
:1064C000E0CFDC01A40FB51F4150504040F0CB019C
:1064D000840F951F2E9105D041505040D8F7089554
:1064E000262FF999FECF92BD81BDF89A019700B48D
:1064F000021639F01FBA20BD0FB6F894FA9AF99A2D
:106500000FBE08950396272FECDFEADF252FE9DF82
:10651000242FE7CF0196272FE4DFE2CFDC01CB0168
:1065200002C02D9105D041505040D8F70895262F34
:10653000F999FECF1FBA92BD81BD20BD0FB6F89468
:10654000FA9AF99A0FBE01960895F894FFCF501069
:1065500076107C1076107C10CE10EF107C10F511A8
:106560000212331C9B1C3B1C051C091C3F1C0D1CF0
:10657000431C4F1C191C941C1D1C531C211C571C14
:106580007C1C251C5B1C831C2B1C611C691C111CA6
:10659000471C151C4B1C2F1C651C731C8C1C921C4F
:1065A000FF1B371CA21CD11BD71BBF1BC71BDD1B2E
:1065B000E31BE91BC21CD91CDD1CE11CE51CE91C0A
:1065C000ED1CF11CF51CF91CFD1C312E4C2E532E1C
:1065D000312C312C862E972EAA2EEB2EF02E312C1C
:1065E000312C312CF82E1F2C232C542C602C6B2C8E
:1065F000762C792CB22CD42C1C2C1C2EDB2CDE2CD3
:10660000E12C0C2D482D4A2D4C2D802D002F0E2FC6
:0E661000252F5A2F772F312C312C9A2FB32F94
:10661E00010F101112131415161718EF0A770D8D9E
:10662E000D6B0B920D6E0D0000010001F13ED5B306
:10663E008BAF7A530044226D3B011901AC0041022D
:10664E005A027A020001020202020606060909092E
:10665E000909090F0F0F0F0F0F0F0F0F0FF7F49000
:10666E00333767F5F1F066363534979695939291F8
:10667E00E200E900EA00B500B600B700CD008301E4
:10668E00CC008A01920194012102230224022502E8
:10669E00260227022A02B300B4006F0070009F0189
:1066AE00CB019F02A002E200E900EA00B500B600AD
:1066BE00B700CD008301CC008A0192019401210222
:1066CE00230224022502260227022A02B300B40066
:0C66DE006F0070009F01CB019F02A00222
:00000001FF
